:020000040800F2
:100000000080002075B00008E1B40008E3B40008E7
:1000100000000000000000000000000000000000E0
:10002000000000000000000000000000E5B400082F
:100030000000000000000000E7B40008CD840008C4
:10004000A9B00008ABB00008ADB00008AFB0000820
:10005000B1B00008B3B00008B5B00008C5BB0008D7
:10006000B9B000080D850008BDB00008BFB0000899
:10007000C1B00008C3B00008C5B00008C7B0000890
:10008000C9B00008CBB00008CDB00008CFB0000860
:10009000D1B000082D850008D5B00008D7B0000801
:1000A000D9B00008DBB00008DDB000081D850008ED
:1000B000E1B00008E3B00008E5B00008E7B00008D0
:1000C000EDAF16204A62304029BD56B31544E9BF52
:1000D00077900D9CFE0B88C07E2615FA83807340B6
:0800E0000FCE674B80D541C033
:1000E800000000000000244000000000000059400B
:1000F800000000000088C3400000000084D797413A
:100108000080E03779C34143176E05B5B5B893460B
:10011800F5F93FE9034F384D321D30F94877825AD7
:080128003CBF737FDD4F15752C
:1001300001000000000000000A00000000000000B4
:100140006400000000000000E80300000000000060
:100150001027000000000000A08601000000000041
:1001600040420F0000000000809698000000000050
:1001700000E1F5050000000000CA9A3B0000000005
:1001800000E40B540200000000E87648170000006D
:100190000010A5D4E800000000A0724E180900006D
:1001A00000407A10F35A00000080C6A47E8D030040
:1001B0000000C16FF286230000008A5D784563016C
:1001C000000064A7B3B6E00D0000E8890423C78AE5
:1001D00010B50124200207490A6802430A6020463C
:1001E00000F00AF8002801D0012010BD08F058F9ED
:0801F000002010BD00200240B8
:1001F800B0B505460E4801780124002916D07D20A7
:10020800C00009F04BFC01460A48006809F046FCAA
:1002180000F02EFE032D09D8002807D10024E04362
:100228002946224600F0ECFD034805602046B0BD93
:0C023800280000202400002014000020FA
:100244000348007803490A68101808607047C046DC
:08025400280000202C0000200E
:0C025C00014800687047C0462C000020DC
:10026800B0B50446FFF7F6FF0546601C02D0044807
:1002780000780419FFF7EEFF401BA042FAD3B0BD87
:04028800280000202A
:10028C00F0B587B0044600200690002C75D0059080
:10029C00A06D002807D125465435204604F0DAFA23
:1002AC0000202870E06501273D072668B068C00073
:1002BC0027D4B0687D4901402943B1607C4800686F
:1002CC007C4909F0E9FB4000801C06900698002848
:1002DC0017D00698401E06900698002811D0069854
:1002EC00401E0690069800280BD00698401E0690DB
:1002FC000698002805D00698401E069006980028FF
:10030C00E7D1B068284208D1A06D10210143A16546
:10031C00E06D012105910843E065B06804210140BE
:10032C00A26D102002405118A26D29D103900F200C
:10033C00C3430493F33B1A40921CA265B268D207E4
:10034C0076D1019027462037226B531E9A41150314
:10035C00A268237E9B031343627ED1031943A27EC2
:10036C0050030843E36803432B430121C807256965
:10037C00002D009009DA854308E0012007B0F0BD9C
:10038C000243A265384607B0F0BD4D052B43387BC0
:10039C0045001D4338780128029109D1002A11D05B
:1003AC00A06D20210143A165E06D02990843E06531
:1003BC00636A002B0BD0072080010340A26A1A430A
:1003CC002A4305E008040543636A002BF3D12A464F
:1003DC00F068394901401143F160032082076368DA
:1003EC001D461540387F0128E76C0AD1206C616CE2
:1003FC000143A06C0843284338430299084305463F
:10040C0000E03D4330692D4901402943316100989A
:10041C00834201990CD093420AD002988007834200
:10042C0006D08804034026490A688243D018086025
:10043C00706907229043656B284370617069702165
:10044C008843A16B09010143716127690123580598
:10045C00874205D0002F0ED1B06A0499084309E0F9
:10046C00B06AE06980001C301C210140049F8F4061
:10047C00206E3843B06270691040A8420AD1002047
:10048C00E065A06D0121014302208143A16505981F
:10049C0007B0F0BDA06D0399084302218843A06505
:1004AC00E06D1843E065012007B0F0BDE8FFFF6F79
:1004BC0024000020400D03000102DEFF02FCFF1FA0
:0404CC0008270140BC
:1004D00070B505460068816882680024D20726D07E
:1004E0000222114023D1816805220A40012A16D137
:1004F0008168104A0A40911C816003210160FFF766
:10050000ADFE064628688068C00710D0FFF7A6FE3B
:10051000801B03282868F6D38168C907F3D0A86D2B
:1005200010210143A965E86D01242043E8652046B8
:0805300070BDC046E8FFFF7F2B
:10053800F0B581B005460024009400688168C907B9
:100548001CD181682D4A2F3211420AD0A86D102182
:100558000143A965E86D01242043E865012001B045
:10056800F0BD8168254A114001273943816024483C
:100578000068000205D4687E012825D1204601B014
:10058800F0BD20480068204909F088FA401C009016
:1005980000980028EFD00098401E0090009800288E
:1005A800E9D00098401E009000980028E3D00098F9
:1005B800401E009000980028DDD00098401E009052
:1005C80000980028E7D1D6E7FFF744FE06462868DA
:1005D8000168C907D2D18168C90704D18168074A6F
:1005E800114039438160FFF735FE801B03282868D6
:1005F800EED30168C907EBD1A8E7C046E8FFFF7F43
:0C0608000827014024000020400D0300E2
:10061400F0B581B00468A56802236D071FD4542582
:10062400455D012D1BD00091174605465435012622
:100634002E70E268D2070BD1A268D20704D0A26858
:100644001B4B13409A1CA260E26801231343E3602E
:100654000446FFF76FFF01230028009E02D01846CE
:1006640001B0F0BDA06D1349014018020818A0653F
:100674000020E06521681C220A602870206D0E4A63
:100684000E4B0F4DC562036342634A681023134344
:100694004B60403132463B4600F0B8FC03462068CC
:1006A4008168034A0A40111D8160184601B0F0BDFB
:1006B400E8FFFF7FFEF0FFFF65B100085BB10008B3
:0406C40049B8000829
:1006C800F0B589B00246002408945420105C012833
:1006D80002D1022009B0F0BD15465435012028701A
:1006E80013689E68760716D416694F68022F9148DA
:1006F80018D10422164386426AD18D48C0430E6839
:10070800F1430143986A084098620020002E63D4A0
:100718002C7009B0F0BD916D20230B4393652C70AC
:1007280009B0F0BD079704273E438642804E60D14A
:100738000A681640986A30431646986230025A6929
:100748008243896801407C48084010435861002072
:10075800002EDDD5012379490F68072189053A461E
:1007680007910A40764906968E4200D082E0D90564
:100778003E460E407ED1714F3868079B984302432E
:100788000A433A6071480068714909F087F90C21F9
:1007980041430C31089108980028B9D000200899E5
:1007A800491E089108990029B2D00899491E089154
:1007B80008990029ACD00899491E08910899002980
:1007C800A6D00899491E089108990029E7D19FE702
:1007D8000E680020002E9BD558490A68594B9E4246
:1007E80067D0594B9E4261D0554B9E4290D105230C
:1007F80060E002971F27079807400F200190059790
:10080800B840176E039087430497086830420690F3
:1008180049D0C00726465DD1069EB00755D470075B
:1008280055D4300755D4F006029E53D4069EB00620
:1008380066D4700666D4300666D4F00566D4B00572
:1008480066D4700566D4300566D4F00466D4B00466
:1008580066D4700466D43004019E3BD40698C00365
:1008680062D40698800361D406984003C017122604
:1008780006402FE03349069E8E4202D119068A426D
:1008880007D331498E4200D042E799050F4000D086
:100898003EE72A4F3E68079B9E4332430A433A602D
:1008A8002C7009B0F0BD4000C60E13E00323DB0531
:1008B80001E003239B051A4007239B050E689E430E
:1008C800B2180A602C7009B0F0BD012602E00226B9
:1008D80000E00326059FBE40049806431666079865
:1008E8008008D269824209D90398C0439A6A0240B3
:1008F800069EB000000FB84010431EE7069E1DE795
:100908000526E7E70626E5E70726E3E70826E1E701
:100918000926DFE70A26DDE70B26DBE70C26D9E701
:100928000D26D7E70E26D5E71026D3E71126D1E7FF
:10093800FFFF07000400008000FFFF0708270140B1
:10094800001000B0004000B8002000B424000020CF
:04095800400D03004B
:10095C00F0B589B00446002708975420205C012884
:10096C0002D1022009B0F0BD26465436012535705F
:10097C002046FFF7A7FD21688A68D207A36D3FD1F7
:10098C000390812252009343981CA065C868CA68E2
:10099C00DD4B1340CB608A68DC4B1A40D2181832FE
:1009AC008A60DB4A024002920846B4300690D94A6B
:1009BC008B68002B2BD5089B5B1C0893089B9342E0
:1009CC0000D996E18B68002B21D5089B5B1C089302
:1009DC00089B934200D98CE18B68002B17D5089BA0
:1009EC005B1C0893089B934200D982E18B68002B17
:1009FC000DD5089B5B1C0893089B9342D8D978E1D2
:100A0C0010210B433770A365004609B0F0BD069862
:100A1C00036888680596F74E30403018059E1830EC
:100A2C0088607F20049003408868002824D50898AB
:100A3C00401C08900898904200D95AE18868002818
:100A4C001AD50898401C08900898904200D950E19B
:100A5C008868002810D50898401C08900898904287
:100A6C0000D946E18868002806D50898401C0890F3
:100A7C0008989042D8D93CE10698006801978F6895
:100A8C00DC4E3740F719059E18378F60019F009593
:100A9C00049D2840009DC3188868002824D5089818
:100AAC00401C08900898904200D922E188680028E0
:100ABC001AD50898401C08900898904200D918E163
:100ACC008868002810D50898401C08900898904217
:100ADC0000D90EE18868002806D50898401C0890BB
:100AEC0008989042D8D904E1069800688F68C14EE6
:100AFC003740F719059E18378F60019F049D2840D9
:100B0C00009DC3188868002824D50898401C0890BC
:100B1C000898904200D9ECE0886800281AD508980B
:100B2C00401C08900898904200D9E2E088680028A0
:100B3C0010D50898401C08900898904200D9D8E02D
:100B4C008868002806D50898401C089008989042A0
:100B5C00D8D9CEE0069800688F68A64E3740F719B2
:100B6C00059E18378F60019F049D2840009DC31877
:100B7C008868002824D50898401C08900898904252
:100B8C0000D9B6E0886800281AD50898401C08904F
:100B9C000898904200D9ACE08868002810D50898D5
:100BAC00401C08900898904200D9A2E08868002860
:100BBC0006D50898401C089008989042D8D998E01F
:100BCC00069800688F688B4E3740F719059E1837CA
:100BDC008F60019F049D2840009DC31888680028E1
:100BEC0022D50898401C08900898904200D980E0C3
:100BFC008868002818D50898401C089008989042DE
:100C0C0077D8886800280FD50898401C0890089859
:100C1C0090426ED88868002806D50898401C089029
:100C2C0008989042DAD964E0069800688F68714E93
:100C3C003740F719059E18378F60019F049D284097
:100C4C00009DC3188868002821D50898401C08907E
:100C5C00089890424DD88868002818D50898401CF0
:100C6C0008900898904244D8886800280FD50898B6
:100C7C00401C0890089890423BD88868002806D5FC
:100C8C000898401C089008989042DBD931E00698EF
:100C9C0000688F68574E3740F719059E18378F60DC
:100CAC00019F049D2840009DC3188868002833D5F7
:100CBC000898401C0890089890421AD88868002818
:100CCC002AD50898401C08900898904211D888683A
:100CDC00002821D50898401C08900898904208D804
:100CEC008868002818D50898401C089008989042ED
:100CFC00DBD93770A06D1021014302208143A1651F
:100D0C00284609B0F0BDC046FC7FFFFFE8FFFF7F1F
:100D1C0003800000FFF10200069800688A68354DD8
:100D2C002A4001252A438A60049A1040C018C00842
:100D3C0000900869800F29D10F2080042E4B1B686E
:100D4C0003409B0C072B21D3D81E01238340079310
:100D5C000798400807900798002817D00798401E5E
:100D6C0007900798002811D00798401E0790079805
:100D7C0000280BD00798401E07900798002805D034
:100D8C000798401E079007980028E7D1069B186823
:100D9C00049A9043009A104318608868154A1040D2
:100DAC000222049210438860FFF752FA06902068E2
:100DBC008168C90713D0FFF74BFA0699401A03282C
:100DCC002068F5D38168C907F2D0A06D10210143CA
:100DDC00A165E06D2843E065284609B0F0BDC16807
:100DEC00029A1143C160A16D01230B430498834304
:0C0DFC00039807E6E8FFFF7F082701408E
:100E0800002805D40322034693430A4A9A1803E0AC
:100E18000C220240064BD2188007C00E8901C9B2C5
:100E28008140FF238340106898430843106070474F
:080E380014ED00E000E400E00D
:100E4000002805D41F21084001218140014801608C
:080E50007047C04600E100E01C
:100E5800002809D41F21084001218140034801606E
:100E6800BFF34F8FBFF36F8F7047C04680E100E03C
:100E7800401E010E01D0012070470749074A506003
:100E8800074803680B4003218907591801600020AF
:100E98009060072111607047FFFFFF0010E000E03D
:040EA80020ED00E059
:100EAC00B0B5002813D00446407F002803D120772A
:100EBC0020460AF060F9022060772079002808D0DB
:100ECC00A168E26820460AF009F9002808D0012040
:100EDC00B0BD20680F49416181681822914381603F
:100EEC0000256079002801D0216900E0E9432068E1
:100EFC00016181686022914362690A438260816862
:100F0C0080229143A2690A4382600120607700200D
:080F1C00B0BDC046B71DC104C1
:100F2400F0B583B0002840D004460646243602209B
:100F34007070276838683049014039602F48803024
:100F4400A0642F483818142108F0AAFD80002B490A
:100F54004118206401916164FC2038400838142150
:100F640008F09EFD1F210140012528468840E064C9
:100F7400E16822690A4361691143A2690A43E1698C
:100F84001143226A0A43A1683B6813430B433B6045
:100F94000295AA0391421B4A0AD1002301990B60CE
:100FA400636010601F461D461BE0012003B0F0BDC6
:100FB40063683F211940019D29601060581E002379
:100FC40003281F461D460CD8481E81005318DD67B0
:100FD40003210140029D8D400B4805607C33BC32E7
:100FE40017460020E06323656765A56530700299A4
:100FF400717003B0F0BDC0460F80FFFF00080240CF
:0C100400F8FFFDBF8408024044090240D0
:10101000F0B582B004462420205C012802D10220D1
:1010200002B0F0BD174625462435012028706A78A5
:10103000012A2ED1022068700020E06325682A680A
:1010400001260196B2432A60A26CE66C5660226DBE
:101050000092002A02D0626DA66D5660226C1C269A
:101060001640019AB2401C4E366816431A4A166062
:101070006B60A368102B3A4600D00A46AA60102B7A
:1010800000D03946E9602968226B002A07D00E2279
:101090000AE0002129708021E16302B0F0BD042242
:1010A000914329602A680A211143296001990902A4
:1010B000626C1368DB0302D513680B431360009B5B
:1010C000002B02D01A680A431A602968019A11435A
:0C10D000296002B0F0BDC04604000240E0
:1010DC00F0B585B03649091F0E68026813680425FF
:1010EC0002932B405F425F410490046C1C2323400D
:1010FC00294699400C46039634406042604138437F
:10110C0031D0019201210227029E304638404442E0
:10111C0044419F40039D2F420A4600D0214604982B
:10112C000446243400292FD008200640774277410A
:10113C00DD40280700D53A46002A23D1019A1068D1
:10114C000E218843106001252946994018480268F1
:10115C000A4302600498C563002121706570416BDD
:10116C0000290ED10EE01068800602D41068A84346
:10117C0010600F4A1068084310600498016B002936
:10118C0000D0884705B0F0BD019B1968890605D4CD
:10119C001A680A218A431A600121617000212170AA
:1011AC00034A116839431160C16A0029E9D1E9E7A2
:0411BC0004000240E9
:1011C000F0B589B0674D2C78012C02D1022009B00E
:1011D000F0BD05900293049203910020079068608F
:1011E0000120287006900704FFF738F806465E4A8B
:1011F0001068C0030AD57D20C400FFF72FF8801BBC
:10120000A04230D2584A10683842F6D11068574987
:101210004B1C1360084002D06860069F9DE001935C
:101220000120069080040890106840030BD57D20B3
:10123000C400FFF713F8801BA04214D24A4A10687A
:1012400008990842F5D10598012850680DD101216F
:1012500008435060039904980860BFF36F8F0298A9
:101260004860144646E0032777E008990843506039
:10127000EFF31080029072B6079A1146039B049E0A
:10128000705858505818741865684560A56885608E
:10129000E568C5602569056165694561A569856180
:1012A000E569C561256A0562656A4562A56A856268
:1012B000E56AC562256B0563656B4563A56B856350
:1012C000E46BC4630F201043403110323F28D7D362
:1012D00025490868384208D00868384205D00868AF
:1012E000384202D008683842F3D1029880F310885F
:1012F0001C4D0C46FEF7B2FF0646206838422246D7
:101300000AD07D20C400FEF7A9FF801BA0421ED298
:10131000154A10683842F6D11068019911601349D6
:10132000084002D06860069F13E010680027089903
:1013300008420ED07D20C400FEF790FF801BA04223
:1013400005D2094A106808990842F5D101E003273F
:10135000054A5068059988435060079828703846B8
:1013600009B0F0BD100F002010200240FA830000E9
:10137000F0B581B0054601200090FEF76FFF0646EC
:10138000254F3868C00318D500980404681C11D094
:10139000FEF764FF801BA8423AD238682042F7D19A
:1013A0000BE03868204208D03868204205D0386801
:1013B000204202D038682042F3D1386817494A1CCD
:1013C0003A60084004D016494860009801B0F0BD6A
:1013D0003968490301D401B0F0BD01218C04691CB6
:1013E00012D00090FEF73AFF801BA84210D2386856
:1013F0002042F7D1E9E739682142ECD0396821422F
:10140000E9D039682142E6D039682142F3D1E2E7D8
:10141000032001B0F0BDC04610200240FA83000056
:04142000100F002089
:101424000648C168002901D40020704704490160BE
:1014340004490160C068C00F7047C04608200240DC
:0814440023016745AB89EFCDE0
:10144C00F0B581B001200090FEF702FF0446194D63
:10145C002868C0030BD5009807047D20C600FEF752
:10146C00F7FE001BB0421AD228683842F7D1286820
:10147C0011494A1C2A60084002D0104948600EE00D
:10148C00286840030BD5009887047D20C600FEF722
:10149C00DFFE001BB04202D228683842F7D1009818
:1014AC00C0076968014369606868C043C00F01B038
:1014BC00F0BDC04610200240FA830000100F00203F
:1014CC0006488168490001D4012070470449016035
:1014DC000449016080684000C00F70470C20024036
:0814EC003B2A19087F6E5D4CDC
:1014F400F0B581B001200090FEF7AEFE0446194D10
:101504002868C0030BD5009807047D20C600FEF7A9
:10151400A3FE001BB0421AD228683842F7D12868CB
:1015240011494A1C2A60084002D0104948600EE064
:10153400286840030BD5009887047D20C600FEF779
:101544008BFE001BB04202D228683842F7D10098C3
:1015540080076968014369606968014048424841FD
:1015640001B0F0BD10200240FA830000100F0020EB
:10157400F0B583B004462C4F3878012802D10220FC
:1015840003B0F0BD019100267E60012038707D20FB
:10159400C5002846FFF7EAFE002802D03E7003B0DB
:1015A400F0BD0420606020680428204B0AD1204844
:1015B400801C1968014319602846FFF7D7FE3E7066
:1015C40003B0F0BDF143019801600021A668E06812
:1015D40080198642009108461DD20295F7001868CA
:1015E400144908403843124908431D4618600298BC
:1015F400FFF7BCFE00280AD1A068E1680818083784
:10160400761C86422B46EAD30098074F03E00199E3
:101614000E60054F2B461968022291431960009E03
:101624003E7003B0F0BDC046100F002014200240ED
:081634000200010005E0FEFFC9
:10163C00F0B581B0354D2978012902D1022001B0D5
:10164C00F0BD00266E600121009129700168CA0767
:10165C002F4F0BD04168012901D0102100E00C2143
:10166C008268C3681B0413437B50016806220A403E
:10167C00062A0BD1014610310EC90B43FF208243C1
:10168C00C143514038680840184323E08A070DD401
:10169C00490720D54169FF229143D2434A403B6818
:1016AC003968DBB2AA2B0DD11C460CE03968194AFB
:1016BC000A40FF21C94351403B680B400069184365
:1016CC00104307E0BB241140CC2B00D1CC24806903
:1016DC002043084338607D20C4002046FFF742FEBB
:1016EC00002802D02E7001B0F0BD009846040C3FCB
:1016FC003868304338602046FFF734FE3968B14310
:10170C000026024D39602E7001B0F0BD100F002084
:08171C002020024000604F078D
:1017240010B5072101604168012901D0102100E0B2
:101734000C210D4A8B583F241C408460895889022F
:10174400890EC16009494161136812680A408261C7
:10175400D9B2AA2901D10A4603E0BB22CC2900D17F
:10176400CC22026110BDC0462020024000604F0719
:10177400F0B58AB00E4609900968002900D1B6E098
:101784005C48099A824201D0052000E003200090C1
:10179400002207921746089203960FE02943196026
:1017A400521C31680846D040089B08330893079BB5
:1017B4001B1D0793BF1C002800D198E0012005469B
:1017C400954029400491EBD0019003231846B8407A
:1017D400C0437468214619404E1E012E069002949F
:1017E400059710D8099B9B6803400398C66809981D
:1017F400BE401E438660E306DB0F93404668AE435B
:101804001E43466003E0032901D1039E1DE0099CA9
:10181400E36806980340039EB568BD401D43E56038
:101824000229029C11D11C20079908400F218140F4
:10183400D3089B00099CE3181D6A8D4331698140DC
:10184400294319627468032121403D46B940099F28
:101854003B68069803400B433B60A0032F46800F70
:101864009ED00320114681432348401805210907CF
:10187400099B8B42016E0BD0214B099D9D4205D0E3
:10188400204B9D42009E04D1022602E0019E00E00E
:1018940000261823089D2B400F259D40A943603046
:1018A4009E400E43066014480168039E7068C3029C
:1018B40002D5049D294301E0049DA9430E4B196000
:1018C4005968830201D5294300E0A9430A4B5960B2
:1018D4000A494968830301D5294300E0A943074B1A
:1018E40059601968C00300D558E7A94357E70AB0FF
:1018F400F0BDC046000C00500018024080180240A1
:0819040000040050000800502F
:10190C00B0B50446074D2868204203D02C60204611
:10191C0009F037FC6868204203D06C60204605F063
:08192C00D1FEB0BD0C18024011
:101934000120000202490A6802430A607047C04657
:0419440000700040EF
:101948000120000202490A6882430A607047C046C3
:0419580000700040DB
:10195C00F0B581B00146032460021B4D2A46143AAF
:10196C00136883430B43136001277A0200209142D2
:10197C0024D1164909682A6852051FD5BE020622D1
:10198C004A4313490090104608F086F80146009827
:10199C00791A022914D02A6832420FD001290FD0AB
:1019AC002A6832420AD000290AD02A68324205D06D
:1019BC00091D032904D02A683242EAD101B0F0BDD6
:1019CC00204601B0F0BDC046147000402400002039
:0419DC0040420F0076
:1019E000F0B587B004460120002C00D1F0E104904E
:1019F0002078C007F74E05943FD12078800761D446
:101A000005980078000700D58FE0059A1078400708
:101A100000D5A0E0D469002C00D1C0E1B068382125
:101A20000140102900D00BE1012C00D1A0E0F068AA
:101A3000032101401346126A914200D098E07021C0
:101A400001405A6A914200D092E07F210902014090
:101A50009A6A1202914200D08AE01F214904014093
:101A6000DA6A914200D083E0072149070840196BE8
:101A70008842049800D0ABE191E1B168F26803209C
:101A80000346934338220A4010215140CB18594253
:101A90005941082A57D0002955D13168636801247B
:101AA000670422049342039008D005252D04AB421D
:101AB00000D0F7E0A304194331603168114331606D
:101AC000059CF8E0B0683821014010204840F268D9
:101AD0000324224002235340C018424242410120C5
:101AE0008702002947D0002A45D103943168059C1C
:101AF000E268002A00D1EDE00722D2029143226978
:101B00000A4332600002316801433160FEF7A6FBF0
:101B100005463068384200D0EEE0FEF79FFB401BE0
:101B20000228F6D9039807B0F0BDB068382101400B
:101B30001829306E49D1800700D466E7059880697E
:101B4000002815D061E73068800300D455E760684D
:101B500000280DD051E7B0683821014020294AD132
:101B6000F06D800700D455E79068002800D051E759
:101B7000049807B0F0BD32683A42059B03D0DA689A
:101B8000002A00D124E101257F20000272688243EF
:101B9000586900021043706000290DD10720C0026F
:101BA0003168814318690843306030688004400F11
:101BB0009549C1409548016095480068FEF71CFBB7
:101BC0000028284600D003E11AE705998969002911
:101BD00000D19AE0012108433066FEF73FFB05463D
:101BE000306E800700D510E7FEF738FB411B03205D
:101BF0000229F5D9ECE0012003900107F06B0840C1
:101C0000029006D1F06B0843F063F06B0840069039
:101C1000069801917F4F3868C00533D403980402B9
:101C2000386820433860FEF719FB054638682042C3
:101C300028D1FEF713FB411B03200229F6D9C7E088
:101C400001210A06306803929043306004914F06E8
:101C5000FEF704FB0546022C09D13068384274D0E7
:101C6000FEF7FCFA411B03200229F6D9B0E03068E8
:101C7000384200D18FE0FEF7F1FA411B0320022920
:101C8000F5D9A5E0F06D05998968012906D00529E7
:101C900000D087E004210843F065F06D0399084304
:101CA000F06588E091433160A00431688143316080
:101CB000002B059C3AD0FEF7D1FA05463068384231
:101CC00000D09AE6FEF7CAFA401B6428F6D90398BA
:101CD00007B0F0BD000281433160FEF7BFFA054650
:101CE0003068384200D18BE6FEF7B8FA401B022874
:101CF000F6D9039807B0F0BD7F20000271688143D8
:101D000060690002084370607AE60121884330660A
:101D1000FEF7A4FA0546306E800700D475E6FEF79C
:101D20009DFA411B03200229F5D951E0FEF796FAEE
:101D300005463068384200D15FE6FEF78FFA401B57
:101D40006428F6D9039807B0F0BDF0683449014023
:101D5000059A106A0843516A0143906A00020843D9
:101D6000D16A0143106B0843F0603068039908435F
:101D7000306004980007F1680143F160FEF76EFAE5
:101D80000446306838420AD1FEF768FA011B032086
:101D90000229F6D91CE0F06820490140F1600020DA
:101DA00007B0F0BD039A9043F065F06D04229043B4
:101DB000F065002910D0184CFEF750FA0546F06D7A
:101DC000800717D4FEF74AFA411B0320A142F6D937
:101DD00007B0F0BD001002400F4CFEF73FFA054679
:101DE000F06D800706D5FEF739FA411B0320A142AA
:101DF000F6D9EDE702980028059A00D00AE6F06BC4
:101E000001998843F06305E60024F40024000020D3
:101E1000140000200070004088130000FCFFFEEF5B
:041E20008C80C11FD2
:101E2400F0B583B00D4601460120002961D002912E
:101E340001907348006807273840A84215D27049BA
:101E44000868B843284308606E4CFEF705FA064656
:101E54006B4800683840A84207D0FEF7FDF9801BA4
:101E6400A042F5D9032003B0F0BD029B1868810796
:101E7400654C0CD5410703D5390322680A43226017
:101E84000F21090222688A43996811432160C0071F
:101E94001AD15B4800683840A8422CD958490868D0
:101EA400B84328430860574CFEF7D6F90646544811
:101EB40000683840A8421ED0FEF7CEF9801BA0422D
:101EC400F5D9032003B0F0BD596803296AD8880006
:101ED40001A2125801989746ED1E00089D1F0008A4
:101EE400891F0008951F00082246083A1268520507
:101EF4005CD403B0F0BD029A10784007424C05D57B
:101F0400380321688143D068084320602068800634
:101F1400400F1FD038212068084008283B4820D0B3
:101F240022680A40102A5AD1616803220A40032A0F
:101F340000D0374861684906490F491C07F0B0FDD5
:101F440061684904490E48436168490F491C07F018
:101F5400A7FD06E02046083800688004410F2C489D
:101F6400C840216889093C220A402A4989581F220D
:101F74000A40D0402849086028480068FEF73AF92A
:101F840003B0F0BD2246083A12689201B1D50DE0C3
:101F9400A26D9207ADD509E02246083A1268920371
:101FA400A7D503E0606D80070198A2D52068B843E7
:101FB40008432060FEF750F90646206838210140A6
:101FC40002984068C000814200D162E7FEF744F9FC
:101FD400801B0C498842F0D9032003B0F0BD20686F
:101FE4000840202802D10120C003BAE72068084035
:101FF400182801D00020B4E77D200002B1E7C046D4
:1020040000200240881300000810024000127A00E9
:102014000024F4007CAF00082400002014000020F9
:1020240010B51E4C20688006400F06D03821206869
:10203400084008281A4807D110BD083C20688004CD
:10204400410F1848C84010BD22680A40102A15D113
:10205400616803220A40032A00D0124861684906D5
:10206400490F491C07F01CFD61684904490E4843A7
:102074006168490F491C07F013FD10BD2068084032
:10208400202802D10120C00310BD20680840182870
:1020940001D0002010BD7D20000210BD08100240B8
:0820A40000127A000024F40090
:1020AC000648006806490968890A1C220A40054945
:1020BC0089581F220A40D0407047C0462400002097
:0820CC0008100240BCAF00083F
:1020D400F0B587B0074680788007564E01D40020BB
:1020E40050E00597012319073246183A1068084052
:1020F400049006D1106808431060106808400690E8
:1021040006980292039101931F024B4C20683843B6
:102114002060FEF7A1F80546206838420AD1FEF790
:102124009BF8401B0228F7D90320059F0499002936
:1021340023D027E0032000900102B0680840059FE7
:1021440011D0B96988420ED0B06801990904B26807
:102154000A43B260B2688A43B2600146374A11400A
:10216400B160C00755D1B06834490840B96901432A
:10217400B16000200499002904D1029B1968039AD4
:10218400914319603968CA0707D18A070DD48A06B2
:1021940013D401224B041AD428E0326803239A434F
:1021A4007B68134333608A07F1D532680C239A4362
:1021B400BB68134333608A06EBD5032212033368EA
:1021C4009343FA681A43326001224B040ED53368F4
:1021D4001C4C23407D692B433360631C9D4205D115
:1021E40013043446483C25681D43256009050ED573
:1021F400910303239B0334689C433B691C43346071
:102204008B4204D11104483E32680A43326007B05D
:10221400F0BDFEF721F80546094CB0688007A2D44A
:10222400FEF71AF8401BA042F7D900980499002938
:10223400A3D0A7E75410024000700040FFFCFFFF4A
:0822440088130000FFFFFF3FBB
:10224C0070B500284BD00446064628367078002816
:10225C0006D130701120C0026060204605F0C8FF26
:10226C00022070702068CA21416253214162C1680A
:10227C00490618D4C16880220A43C260FDF7E8FF02
:10228C0005462068C16849060DD4FDF7E1FF401BE7
:10229C007D21C9008842F4D9032070702168CA6876
:1022AC00FF224A6270BD8169174A0A408261A168A7
:1022BC0062690A43E169114382690A4382612169B7
:1022CC000161E168090402690A430261204600F0D9
:1022DC001DF82168002804D0FF224A6270BD01203D
:1022EC0070BD072040078A6982438A61206A626A4E
:1022FC000243A06910438A6902438A61FF20486245
:0C230C0001207070002070BDBFFF8FFB2F
:10231800F0B581B00446234F38460C380168802256
:10232800914301607D20C6003868800615D4206876
:10233800C168A0229143C160FDF78CFF0546206863
:10234800C068800623D4FDF785FF401BB042F6D94C
:1023580029210320605401B0F0BD38682021009184
:10236800884338602068C168A0229143C160FDF7A6
:1023780071FF05462068C06880060BD4FDF76AFF28
:10238800401BB042F6D929210320605403E0002005
:1023980001B0F0BD00203968009A1143396001B0DE
:0823A800F0BDC04618280040FA
:1023B000F0B583B004462820205C012802D1022019
:1023C00003B0F0BD16460D4622462832022050705A
:1023D0002068CA2141625321416201210292019188
:1023E0001170C16849061CD4C16880220A43C260CA
:1023F000FDF734FF07462068C168490611D4FDF790
:102400002DFFC01B7D21C9008842F4D90320029B07
:1024100058702168CA68FF224A620021197003B00F
:10242000F0BD826940211140002E04D00029019E98
:102430003CD1E9703CE0002900D1E9702A78002104
:1024400013460A3B08D3DAB2CD265643F60A0A22CF
:1024500072439A1A360110361643F2B213046A78A0
:1024600016460A3E0F4608D3F2B2CD275743FF0A5D
:102470000A227A43B21A3F0110371743FAB2120206
:102480001A43AB781E460A3E08D3F1B2CD234B4324
:10249000D90A0A234B43F31A090110311943C9B26F
:1024A0000A43E9788B051343019E09E0E978890521
:1024B0002A7812046B781B029A18AB78D3180B4356
:1024C0000C4919400160B10482698A438261E9685C
:1024D0002A690A438169114381612046FFF71CFF85
:1024E0002168FF224A620028029B96D15E70187014
:0824F00003B0F0BD7F7F7F0007
:1024F800F0B585B000280BD005465C3541218E002B
:10250800416A002907D0002101610146143107E022
:10251800012005B0F0BD4168B14203D001461C312D
:1025280000220A60002787626978002904D129708F
:10253800044605F06FFF2046022104950191697059
:1025480001680A6840239A4303910A60C268264BCF
:1025580001259A422B4600D300231B03ED021543A5
:102568000F27390202918D4201D000258562456806
:10257800876835402124A4023C4064190569019903
:102588000D4025434169012421402943FC368769D0
:102598003E400E43C16938250D403543016A802607
:1025A8000E402E436103856A0D403543039E356016
:1025B800390C04250D4002990A4013432B43416A04
:1025C80010220A401A43416B08230B4013437360DF
:1025D800E102F2698A43F261002101660020049950
:0C25E8004C7005B0F0BDC04601070000BB
:1025F400F0B585B0044607464437387E012802D139
:10260400022005B0F0BD1E460292039101253D76DD
:10261400FDF722FE0490797E012900D0A5E00398FD
:10262400002800D141E10298002800D13DE1002EAC
:10263400284600D1A5E0787E042801D005207876CC
:10264400002323667E80E687E1689E4A012001918B
:10265400914200D31D462D03020320684168914333
:1026640049194160029921643E80039DA563E36496
:102674002365A6870168490603D4016840220A43FA
:10268400026061684A424A41711E4B424B41134306
:1026940001998C4A91420A9E77D3002B06D029884F
:1026A400C160A81CA063E08F401EE0870125701C58
:1026B40032D101E0FDF7D0FDE08F002803D1788806
:1026C400002800D1CDE02068816889070DD5E18F0D
:1026D40000290AD0012D08D1A16B0A88C260891C87
:1026E400A163E18F491EE18700258168C907E1D014
:1026F40079880029DED0216CC0680880881C206499
:102704007888401E78800125D4E7FDF7A5FD04995B
:10271400401AB04200D3CDE0E08F002803D178887E
:10272400002800D19DE02068816889070DD5E18FDC
:1027340000290AD0012D08D1A16B0A88C260891C26
:10274400A163E18F491EE18700258168C907DCD0B8
:1027540079880029D9D0216CC0680880881C20643D
:102764007888401E78800125CFE741208200636885
:102774000220934205D1042903D1A168002900D184
:102784004DE70021397605B0F0BD002B07D029783C
:102794000173A06B401CA063E08F401EE0870125FD
:1027A400701C33D101E0FDF757FDE08F002802D102
:1027B4007888002855D02068816889070FD5E18F73
:1027C40000290CD0012D0AD1A16B09780173A06BEB
:1027D400401CA063E08F401EE087206800258168CC
:1027E400C907E0D079880029DDD0007B216C08700E
:1027F400206C401C20647888401E78800125D2E734
:10280400FDF72AFD0499401AB04253D2E08F002804
:1028140002D17888002824D02068816889070FD5E0
:10282400E18F00290CD0012D0AD1A16B0978017325
:10283400A06B401CA063E08F401EE0872068002549
:102844008168C907DCD079880029D9D0007B216C44
:102854000870206C401C20647888401E7880012514
:10286400CEE703200390C10220463246049D2B4646
:1028740000F02AF800280FD1204631462A4600F0FD
:10288400D5F8002808D103984102204632462B4649
:1028940000F01AF8002805D0206E20210843206695
:1028A40021660120216E002905D0012000213976FE
:1028B40005B0F0BD0320012179760021397605B0F9
:0828C400F0BDC0460107000051
:1028CC00F0B587B0049314460D46074605A80026BC
:1028DC000670FDF7BDFC0499081A02940419FDF763
:1028EC00B7FC04904E48006823214143080D604317
:1028FC00069003973F68B868284233D001960320AE
:10290C0046020299491C30D00290B5421CD104E019
:10291C00039800688068304245D0387B05A9087060
:10292C000598FDF795FC0499401AA0423ED20698F2
:10293C000699491E06910028EAD10024E8E703987D
:10294C000068806828422ED0FDF782FC0499401A5A
:10295C00A0422BD206980699491E06910028EED16A
:10296C000024ECE7002007B0F0BDB54247D1387B1E
:10297C0005A908700598B868304214D0387B05A9B1
:10298C0008700598B86830420DD0387B05A90870DE
:10299C000598B868304206D0387B05A908700598B0
:1029AC00B8683042E3D1019807B0F0BD039D2968A7
:1029BC004868E02290434860412080006A68824267
:1029CC0002980BD1AA680123DC03A24202D09B021D
:1029DC009A4203D10A6840239A430A6001225303A6
:1029EC00AC6A5C359C4205D10C689C430C600C684D
:1029FC001C430C60002129706A7007B0F0BD01996E
:102A0C00B868284208D0B868284205D0B86828426F
:102A1C0002D0B8682842F3D1084607B0F0BDC046D2
:042A2C002400002062
:102A3000F0B583B015460E460446FDF70FFC281A84
:102A40008719FDF70BFC05462C4800684001000D76
:102A50007843029021688A680020120622D5721CF1
:102A60001DD0019026465C3603E020688068000691
:102A700041D5FDF7F3FB401BB84215D202980299ED
:102A8000491E02910028F0D10027EEE78A6812065D
:102A900008D58A68120605D58A68120602D58A68A2
:102AA0001206F3D403B0F0BD20684168E0229143E0
:102AB00041604121890062688A420BD1A1680122EC
:102AC000D303994202D09202914203D1016840227D
:102AD0009143016001214A03A36A934205D103682F
:102AE00093430360036813430360002030707170E8
:102AF000032003B0F0BD019803B0F0BD2400002016
:102B0000B0B5002823D005463C356978002904D1AA
:102B10002970044608F0CFFB204602216970016845
:102B20000C682D4B994202D02C4A914211D170224F
:102B30009443826822432A4CA1420EDC274CA142D6
:102B400014D02B4CA14211D099420FD042E0012069
:102B5000B0BD2246224CA142F0DD224B994205D065
:102B6000214B994202D0214B994233D103231B02BE
:102B70009A43036913438022934382691A430A608C
:102B8000C268CA6242688A621A4A8A180A23DA410B
:102B9000072A06D801239340E122134201D042695B
:102BA0000A6303463E33443001224A610C69E4075C
:102BB00002D00C6994430C6102711A705A709A70B9
:102BC000DA701A715A71027042708270C2706A7043
:102BD0000020B0BD1346CEE7002C014000040040A9
:102BE000FF3F0140004001400048014000440140D7
:082BF0000020004000D4FEBFEC
:102BF80070B504463C340221617006463E360546EF
:102C0800443501680A6A0E4B1A4207D10A6A0D4B0D
:102C18001A4203D10A6801239A430A6008F048FB64
:102C28000020287130707070B070F0703071707161
:102C380028706870A870E8702070607070BDC04619
:082C480011110000440400001A
:102C5000F0B582B004463E340346443301270029D0
:102C600019D0019001200E1F02220092D641032E9E
:102C700034D8B50001A77D59AF46C0468D2C000859
:102C8000C92C0008B52C0008BF2C0008671C3F7831
:102C900008291DD126E022781D786D1E6E1EB541D3
:102CA000012A3E4600D12E46002E27D10222227054
:102CB0001A7050E0E71C3F78082909D112E0271D5F
:102CC0003F78082904D10DE0A71C3F78082909D0D6
:102CD000042901D15D1C06E0DD1C04E0671D3F787E
:102CE0000829F5D19D1C2D786D1E6A1E9541012F76
:102CF000074600D12F46002F03D00127384602B0E7
:102D0000F0BD032E074620D80198C0467E44367990
:102D10007600B7440110060B009A627008290ED1A4
:102D200018E0009AE270082909D113E0009A227194
:102D3000082904D10EE0009AA27008290AD00429BB
:102D400001D15A7007E0DA7005E0009A62710198CB
:102D50000829F4D19A7002220B46D341032BCDD817
:102D60009A00144B9B580268D0681843D0601F200B
:102D70000140012318468840116A81431162116A9B
:102D8000014311620C48824205D00C48824202D0B5
:102D90000B48824208D190680A4901400027062961
:102DA000ACD018048142A9D01068184310600020EC
:102DB00002B0F0BD20AF0008000400400040014018
:082DC000002C01400700010096
:102DC80070B502230A46DA41032A2FD89200274C0D
:102DD800A2580468E5681540E5601F250D400122EA
:102DE8001646AE40256AB5432562256A2562256ADE
:102DF8001F4E354206D1256A1E4E354202D125683E
:102E08009543256004463E344430002910D00D1FF8
:102E1800DD41032D23D8C0467D442D796D00AF4494
:102E280001130B0F6270082911D11BE0012070BD3E
:102E380022700270002070BDE270082907D111E0ED
:102E48002271082903D10DE0A27008290AD00429AB
:102E580002D14270002070BDC270002070BD627146
:102E68000829F4D18270002070BDC04630AF000838
:082E78001111000044040000E8
:102E8000F0B583B004460068C5680227294639407A
:102E90004A424A410169029139404B424B41134336
:102EA00013D16A49FE3101610121217780698007D0
:102EB00003D0204600F0F8FE05E0204608F0FDF9BA
:102EC000204608F0FBF9002020770126042229463D
:102ED00011404842484102994907314600D5014610
:102EE000032000020190002916D100922068574962
:102EF000FC310161277780690199084203D020469F
:102F000000F0D2FE05E0204608F0D7F9204608F090
:102F1000D5F900202077009A0827294639404842F1
:102F2000484102990907314600D50146002913D1CD
:102F300020684649F83101612277C069800703D0D3
:102F4000204600F0B1FE05E0204608F0B6F9204624
:102F500008F0B4F900202077102129404842484168
:102F60000299C906314600D50146002914D12068CE
:102F70003649F03101612777C0690199084203D0D1
:102F8000204600F091FE05E0204608F096F9204624
:102F900008F094F900202077012129404842484157
:102FA0000299C907314600D00146002906D12068A0
:102FB0002649FF310161204608F081F980272F4022
:102FC000784278414121C901029A0A42314600D033
:102FD0000146002905D120681D490161204608F0FD
:102FE00071F9784278410299C905314600D5014608
:102FF000002905D1206815490161204608F063F9D0
:10300000402129404842484102994906314600D5AD
:103010000146002906D120680C49C03101612046D3
:1030200008F04EF92020054068426841029989065F
:1030300001D403B0F0BD0600FBD120680349E031A4
:103040000161204608F03DF903B0F0BDFFFEFFFF2F
:043050007FDFFFFF20
:10305400F0B582B03C23C35C012B02D1022002B044
:10306400F0BD03463C330224E241032A00D9A3E025
:103074007A4412795200974401752E4F0268146AFB
:10308400156A012085431562CD68019560C90096D3
:1030940097694D4E0839B24205D04C4EB24202D027
:1030A4004B4EB24202D10320874300980743104697
:1030B4001830F026B743019E3601F6B2BE19966168
:1030C4000A263540B4436419146294690C25AC4350
:1030D4009461896869E00068026A01242402056A2F
:1030E400A54305624C68F025AC43CD682D01EDB2D3
:1030F4002C19C569F326B5432543C561052464022B
:103104000D682D022540A24352190262C2690C24A3
:10311400A243C261896823E00068026A012424038F
:10312400056AA54305624C682402264D2540CC68F7
:103134002403A4B26419F3252D02C669AE432643C1
:10314400C661052464030D682D032540A24352196A
:10315400026203229202C4699443C4618968090229
:103164001C3022E00068026A046A1025AC43046241
:103174004C682402134D2540CC682403A4B264197E
:10318400F3252D028669AE43264386610C6824012B
:10319400A0252C40AA4312190262032292028469D8
:1031A4009443846189680902183002680A43026002
:1031B4000020187002B0F0BD01200021197002B087
:1031C400F0BDC046000FFFFF000400400040014076
:0431D400002C01408A
:1031D8000222D141032915D87944097949008F443D
:1031E800010D0509006834300068704700683C30FC
:1031F80000687047006840300068704700683830E1
:083208000068704700207047C8
:1032100010B53C23C35C012B01D1022010BD034635
:103220003C33002A07D0082A03D0042A0DD10A4AC9
:1032300003E0084A01E00F22D2430068846E144084
:103240000C4384660020187010BD01200021197005
:0C32500010BDC046FFFFF0FFFFF0FFFFC5
:10325C0070B50446026810686F490140A068236984
:10326C00034360691843636E03430B43E1690B43EB
:10327C0013600320000353688343E06818435060D5
:10328C00A069236A03439068644D05401D43956013
:10329C00D36A0F208343606A0343D3620023604DDB
:1032AC00AA4206DC614DAA4212D0614DAA4215D049
:1032BC000CE05C4DAA4211D05B4B9A4206D15D4AA0
:1032CC0012689207120F5C4B9B5807E0102305E025
:1032DC00584A12680C231340574AD358264668366E
:1032EC000125EA03914216D1082B00D989E0C0468A
:1032FC007B441B795B009F4404843684248484843F
:10330C004200FEF7CDFE626A0B2A1FD301210B2A65
:10331C0046D1090244E0082B00D972E07B441B79AA
:10332C005B009F44046E266E176E6E6E3200FEF7C5
:10333C00B7FE626A0B2A12D301210B2A54D109025F
:10334C0052E0FEF769FE626A0B2ADFD291003C4A1A
:10335C00515825E0FEF760FE626A0B2AECD2910010
:10336C00374A515840E00B2815D28000344909588F
:10337C0015E00B281AD280003149095819E00B28A6
:10338C0019D240002D49095A19E00B2827D24000C8
:10339C002A49095A27E001210B2800D109022948A2
:1033AC0006F07AFB400061684A080EE001210B2808
:1033BC002ED0244818E001210B2800D10902E80383
:1033CC0006F06AFB420061684808101806F064FBBE
:1033DC001D49014015D00007400F08430EE00121A4
:1033EC000B2800D10902E80306F056FB61684A0875
:1033FC00101806F051FB80B2102802D32168C86067
:10340C000025124830600020E0662067284670BD19
:10341C0009020C48E8E7C046F369FFCFFFF4FF113F
:10342C00FF4B0040004C004000380140004400407D
:10343C00004800405410024040AF000832B8000869
:10344C0050AF00080024F400F0FF00000100010060
:10345C00F0B581B0044606467C3600200090F06042
:10346C00FCF7F6FE05462168086800070ED5C8690A
:10347C0080020BD401204705FCF7EAFE401B1849DB
:10348C00884221681AD8C8693842F5D008684007C4
:10349C00009A10461DD5C8694002104619D4012067
:1034AC008705FCF7D5FE401B0D498842216805D8DD
:1034BC00C8693842F5D0009A10460AE00D20400148
:1034CC000A6882430A60886801229043886003205E
:1034DC00009A202171603270B16001B0F0BDC0461D
:0434EC00FFFFFF01DE
:1034F000F0B581B004467C3465680223202D12D1DA
:10350000012500290CD0002A0AD0866800952F03D7
:10351000BE420BD1CD0709D00569002D06D1009D13
:10352000284601B0F0BD022001B0F0BD2578012D84
:103530001D46F5D0034654335A800025E5601A80B5
:10354000016521216160009B5907426E8A420BD1BF
:10355000BE4202D10169002916D0104925700167C9
:10356000D9050068083009E0BE4202D1016900298E
:103570000CD00849257001670068802102680A4361
:103580000260002001B0F0BD0349E7E70049F1E720
:10359000FD3500083DBB0008A13500089BB30008BD
:1035A00070B58021415821291AD102465632938A9A
:1035B000002B15D00168104C02E05B1E1D040FD0DB
:1035C0001588002D0DD0CD692D06F6D5056D2E88F8
:1035D00026408E62AD1C056515886D1E1580ECE7D2
:1035E00070BD0120C0058A6882438A600868402255
:0C35F00002430A6070BDC046FF010000ED
:1035FC0030B58023C15821290FD10246563211888B
:10360C00002901680AD0036D1C88084D25408D6285
:10361C00991C01651088401E108030BD08689843C5
:10362C0008600868402202430A6030BDFF010000B8
:10363C00F0B584B004467C34A3680227202B13D148
:10364C00012300290DD0002A0BD0866801252B03FD
:10365C0003939E420BD1CB0709D00369002B06D1F3
:10366C000123184604B0F0BD022004B0F0BD23784D
:10367C00012B3B46F5D003465C335A801A8081659A
:10368C00002E00930FD029078E4207D003998E424B
:10369C0010D1016900290BD125490CE001690029E1
:1036AC0004D03F2107E00169002901D07F2102E00D
:1036BC00FF2100E0002199800023E3602221A1601A
:1036CC000768B96829430197B96029020291690713
:1036DC00476E8F4203D10099898991420CD9039985
:1036EC008E4202D1016900291DD0154A2370C26691
:1036FC0002992031019A10E003998E4202D101699E
:10370C00002912D00C4E019F3A4608322370C6662F
:10371C00386802990843386029071068084310601C
:10372C00002004B0F0BD054AE0E7024EEBE7C046CE
:10373C00FF01000051370008F1370008EDB3000815
:04374C0047B4000876
:10375000F0B581B004468420205822282BD125467C
:103760005E356E89002E2AD02046843000906F8806
:1037700002E0761E300422D02068416A3940A26DF2
:1037800011802988491E2980911CA165298800295A
:10379000EFD10121090202688A4302608168124A5E
:1037A000114081600020E0662020009908602046DA
:1037B00007F079FEDDE72068183008210EE0288840
:1037C00000280ED0698988420BD20848E066064876
:1037D000411C206882680A408260202102680A43F6
:1037E000026001B0F0BDC046FEFFFFEFEDB3000880
:1037F000F0B581B004468420205822282DD12546DA
:103800005E356E89002E2CD02046843000906F8863
:1038100002E0761E300424D02068406A3840A16D52
:1038200008702888401E2880A06D401CA06528884C
:103830000028EED10120000221680A6882430A6054
:103840008868124A104088600020E06620200099B5
:103850000860204607F027FEDBE7206818300821C3
:103860000EE0288800280ED0698988420BD20848CB
:10387000E0660648411C206882680A408260202178
:1038800002680A43026001B0F0BDC046FEFFFFEFD0
:0438900047B4000831
:10389400F0B581B000219C4D0B46009107E0254610
:1038A400E355002B7ED05B1C802B00D181E02C469D
:1038B4009A0094488558802602460F4603E0103E3D
:1038C4004032002EEBD0106885422DDC50688542D2
:1038D4002EDC906885422FDCD068854230DC10698C
:1038E400854231DC5069854232DC9069854233DCA3
:1038F400D069854234DC106A854235DC506A8542E1
:1039040036DC906A854237DCD06A854238DC106B3D
:10391400854239DC506B85423ADC906B85423BDC56
:10392400D06B8542CBDD3BE07F1C50688542D0DD07
:103934007F1C90688542CFDD7F1CD0688542CEDD38
:103944007F1C10698542CDDD7F1C50698542CCDD2A
:103954007F1C90698542CBDD7F1CD0698542CADD1E
:103964007F1C106A8542C9DD7F1C506A8542C8DD10
:103974007F1C906A8542C7DD7F1CD06A8542C6DD04
:103984007F1C106B8542C5DD7F1C506B8542C4DDF6
:103994007F1C906B8542C3DD7F1CD06B85428EDD1E
:1039A4007F1C8CE70098012800D1A6E00123009336
:1039B4007DE7564940240C70002203E01032802A2F
:1039C40000D198E0A85C84422ED0AB185878844289
:1039D40030D09878844233D0D878844236D018795D
:1039E400844239D0587984423CD0987984423FD07B
:1039F400D879844242D0187A844245D0587A844295
:103A040049D0987A84424DD0D87A844251D0187BD8
:103A1400844255D0587B844259D0987B84425DD0EF
:103A2400D87B8442CAD161E00A70D4B2AB1858780A
:103A34008442CED1501C0870C4B298788442CBD151
:103A4400901C0870C4B2D8788442C8D1D01C0870C5
:103A5400C4B218798442C5D1101D0870C4B2587913
:103A64008442C2D1501D0870C4B298798442BFD137
:103A7400901D0870C4B2D8798442BCD1D01D08709E
:103A8400C4B2187A8442B9D1104608300870C4B25E
:103A9400587A8442B5D1104609300870C4B2987A75
:103AA4008442B1D110460A300870C4B2D87A844234
:103AB400ADD110460B300870C4B2187B8442A9D132
:103AC40010460C300870C4B2587B8442A5D110460D
:103AD4000D300870C4B2987B8442A1D110460E30D8
:103AE4000870C4B2D87B844200D067E710460F3018
:103AF4000870C4B262E701B0F0BD054804F0DCFF11
:103B0400FEE7C046FC070020BA130020290000206D
:043B1400CABF00081C
:103B180080B500F07FF802480421016080BDC046EE
:043B28009C0F0020CE
:103B2C00F0B583B000F074F8314F04200290386087
:103B3C003048006800900023304C07E00026019BC1
:103B4C00980032490E505B1C802B45D0294A1068D6
:103B5C002949084001931902401810600BE001201C
:103B6C00386000212046FFF76DF81520FDF762F94B
:103B7C000226022EE3D138680428F0D038680226D9
:103B8C000328F6D138680328D8D11520FDF75EF943
:103B9C00002520462946FFF711F90298386018488D
:103BAC000168002908D0174B1868174A12681203CD
:103BBC0080181860092903D8481C11490860D8E7F7
:103BCC000F490D600F490D600A2105F065FF216852
:103BDC00896A4E1C4643CCE77F200002009A0240C3
:103BEC0004490868044B18401043086003B0F0BD4A
:103BFC009C0F002004100240FF80FFFF540E002099
:103C0C00480F00205C0F0020A00F0020FC070020B4
:103C1C0070B584B0012670041C490A6802430A601E
:103C2C001B4D1C4A2A6009680140009100982846E7
:103C3C00FEF7DCFF184800246C60AC60E8602C6177
:103C4C002846FEF757FF002800D0FEE703940C200F
:103C5C000290019600940E4869460022FFF7F4F991
:103C6C00002800D0FEE70A4802210022FFF7CAFA1A
:103C7C00002800D0FEE7152000210A46FDF7BEF80B
:103C8C001520FDF7E3F804B070BDC04640100240AB
:0C3C9C00540E002000440140FFFF000017
:103CA800F0B581B0017F01293BD11F4E3168012950
:103CB80006D10021FFF78CFA1E49086002202FE088
:103CC800316802292DD100210446FFF781FA174FE8
:103CD80038601520FDF7BCF815480021FFF770F88B
:103CE8000220C0432168086112480068396881428F
:103CF80001D9081A03E0FED2081A0F4940180F49E3
:103D08000860086800030E49884208D20D4804F08C
:103D1800D1FE0A48006801030B4805F08BFF032019
:103D2800306001B0F0BDC0469C0F0020880F002015
:103D3800540E00208C0F0020FFFF0000A00F002071
:0C3D4800405DC600F0C300084EC100083A
:103D5400F0B583B00D46044601600C20404906C509
:103D64000021E86029616961A961E9612962012092
:103D740002900703083D2E467C360998089A002BCA
:103D840004D0012B05D10321490203E002998902E1
:103D940000E00F46AF602961511E4A1E914149035C
:103DA400E96005F0F3FD00272E4B3A4607F0B7FB18
:103DB40005F074FD01907068002803D1377028461F
:103DC40004F03AFC2420706028680168029FB9431B
:103DD40001602846FFF740FA01282AD0A86A002883
:103DE40002D0284607F06EFAF8052E687168014380
:103DF4007160B8063168014331606F680320400286
:103E0400D6307843184905F04BFE18498F42019A81
:103E140000D3421CFF200006716901401143716107
:103E24003068029F384330602846FFF715FB0028AE
:103E340001D007F052FB206807F034FB002801D0C2
:103E440007F04BFB206827343A022146FFF7F4FBC6
:103E5400002803D0064805F0EFFEFEE703B0F0BDEE
:103E64000038014000000C4040420F00014B0000AC
:043E7400E0BF0008A3
:103E7800F0B58DB005460268D16910680C9050689D
:103E880001200A90000709900695803590680B90EC
:103E98000807089049D00998431C0B98034001264D
:103EA80037023C4620340C9804401C433DD0074060
:103EB8007C427C41CF070A9F00D02746002F03D1C0
:103EC8001662AC683443AC600B9806407442744187
:103ED8008F070A98074600D52746002F05D10224E8
:103EE8001462AC6804272743AF60744274414E07DC
:103EF800064605D4002E05D0089800280BD414E0F7
:103F08002600F9D104241462AC6802262643AE6068
:103F18000898002809D520240C980440234304D08D
:103F280008231362AC681C43AC600126F0050790B7
:103F38000B050FD50B9B0340B4060C980440E318FF
:103F480008D0F302136220236B602B605F4B1E7551
:103F58005F4C1E55059620200B460890034004939D
:103F680020D00B9B099803400C9C089804401C43E4
:103F780018D06B68222B11D14523DB00534CE6582F
:103F880005980702BE4209D2A619526A2727F25598
:103F98004F4AA054E258521CE25003E093690824A7
:103FA8001C43946180240E4626400A9835D00B9A0B
:103FB800079B1A400C9B234013432ED0434A136897
:103FC8001A59212A14D11A4656321788002F1F6809
:103FD800039716D01F6D029701923F78039A976254
:103FE800029F7F1C1F65019A13885B1E13800FE0D8
:103FF8001A681368A3431360136840271F431760A8
:1040080006E03A68A2433A603A68402313433B60AB
:1040180023221201059B2D4FBB5440270C9B3B408C
:104028005A425A41490606D4002806D0A8680028F2
:1040380015D10DB0F0BD1000F8D12648002101704F
:10404800069803681A68BA431A60016708992960D4
:1040580007F024FA22206860A8680028E9D0222303
:104068006B600498002807D00B98099901400C98B8
:10407800089A104008431ED1002EDAD00B990798F1
:1040880001400C9820400843D3D026200F4C002133
:1040980021540698222603681A68BA431A600167F1
:1040A8000899296007F0FAF96E6023200001059944
:1040B80021540DB0F0BD06980068816908220A43B2
:1040C80082610020A8600DB0F0BDC046C805002080
:0840D80031020000EE0500209A
:1040E000F0B585B04521CC000159052906D2021949
:1040F000002101751160084605B0F0BD0494272227
:10410000825C00920346273301220C46144003943C
:10411000D5438A1E0192154002935B1C6A4A6B4E7E
:1041200003E0AD1E9B1C002D71D05C1E2478544012
:104130006208E40730D15408D20731D16208E4079D
:1041400032D15408D20733D16208E40734D154087D
:10415000D20735D16708E20736D17A08FC0700D0CC
:1041600072401C7854406208E40732D15408D207E8
:1041700033D16208E40734D15408D20735D162083C
:10418000E40736D15408D20737D16708E20738D19F
:104190007A08FC07C5D038E072405408D207CDD069
:1041A00074406208E407CCD072405408D207CBD0E8
:1041B00074406208E407CAD072405408D207C9D0DC
:1041C00074406708E207C8D077407A08FC07C7D177
:1041D000C7E772405408D207CBD074406208E407A6
:1041E000CAD072405408D207C9D074406208E407AC
:1041F000C8D072405408D207C7D074406708E2079D
:10420000C6D077407A08FC078BD0724089E7039CC0
:10421000002C03D1049C4B1C1FD168E75B1E1B784C
:104220005A405308D207049C2DD15A08DB072ED1DF
:104230005308D2072FD15A08DB0730D15308D207D1
:1042400031D15A08DB0732D15308D20733D15A088B
:10425000DB0734D14B1C00D149E7029D019BEB5C8D
:104260006918491E09780902C918914200D03EE731
:104270000221009B002B00D13DE7154A128B9A4288
:1042800000D034E737E773405A08DB07D0D07240DC
:104290005308D207CFD073405A08DB07CED0724004
:1042A0005308D207CDD073405A08DB07CCD07240F8
:1042B0005308D207CBD073405A08DB07CAD07240EC
:1042C0004B1CCAD113E7C046FFFF000001A000004D
:0442D000300000209A
:1042D400F0B585B0054627202B5CFF242046283006
:1042E4002B544521C9006918002702914F602818F2
:1042F4002946273101260490324600F0E5F80346AA
:104304000395263501950028204600D1A7E01846DC
:10431400304000906A4A6B4D012B05D13C4638462B
:10432400009900297ED19AE01846B043049E03E028
:10433400B61CBF1CB84270D0317869404C08C9071C
:1043440030D16508E10731D16C08E90732D165083D
:10435400E10733D16C08E90734D16508E10735D1A9
:104364006908EC0736D14C08C90700D05440757869
:1043740065406908EC0732D14C08C90733D161089C
:10438400E40734D14C08C90735D16108E40736D1B4
:104394004C08C90737D16108E40738D14D08C9076B
:1043A400C6D038E054406508E107CDD055406C08CC
:1043B400E907CCD054406508E107CBD055406C08E0
:1043C400E907CAD054406508E107C9D055406908D7
:1043D400EC07C8D051404C08C907C7D1C7E75140C2
:1043E4004C08C907CBD054406108E407CAD05140F7
:1043F4004C08C907C9D054406108E407C8D05140EB
:104404004C08C907C7D054406108E407C6D05140DE
:104414004D08C9078CD055408AE7280A2C460099D4
:1044240000291CD00498C05D45406808E9072AD1DA
:104434004108C0072BD14808C9072CD14108C0073F
:104444002DD14808C9072ED14108C0072FD14808EB
:10445400C90730D14408C00700D05440200A049949
:10446400CC54CA1850700C20019A10709A1C029DEA
:104474006A60039C206892B2FFF738F80020286035
:10448400207505B0F0BD50404108C007D3D051405D
:104494004808C907D2D050404108C007D1D0514084
:1044A4004808C907D0D050404108C007CFD0514078
:1044B4004808C907CED050404408C007CDD1CDE745
:0844C40001A00000FFFF000051
:1044CC00F0B586B04C78102C1CD0062C0BD0032CDD
:1044DC0027D1894C248B002B3BD09C4239D0862190
:1044EC0081540B2181E0844C258B002B01D09D4203
:1044FC000ED1CD788B781E027619B708772F36D36C
:10450C0086215AE07C4C258B002B13D09D4211D078
:10451C008621815480180B2141700220801806B02E
:10452C00F0BD80214C408454801801214170901CB6
:10453C0006B0F0BD4F790B791B02DB191D467C3D93
:10454C007B26F643B54229D890218154801803214B
:10455C00E2E74E790B791B029C1923467E3B7D27A3
:10456C00FF43BB4230D88321815403213DE07600C8
:10457C000496A71905970F79059E77704F79049EBD
:10458C00A755062484548018857043700B79C3702A
:10459C00497901710520801806B0F0BD0390049292
:1045AC00CA788C782502AE189819544BC5186D1E14
:1045BC009D421FD29021049A0398815480180221A5
:1045CC004170881806B0F0BDCB7889780591090246
:1045DC000393CB188118E418484FE7197F1E474DF9
:1045EC00AF4242D283230B70022180184170901C81
:1045FC0006B0F0BD02970092530001946502EB18CF
:10460C003D4AD318059300251A4653194C19E779DE
:10461C005F70277A5755771C874215D2677ADF70FF
:10462C00A77A9F70B71C87420ED2E77A5F71277BFF
:10463C001F71F71C874207D2677BDF71A47B9C71CB
:10464C000835361D8642E0D31021049A0398815414
:10465C008018029901710021C17000998170019933
:10466C0041700520801806B0F0BD032704928754D2
:10467C007000487003984000059A560230181E4A84
:10468C001018059000200A460E182546059C271880
:10469C007978B170215CF170591CA9421CD22C465E
:1046AC00F9783171B9787171991CA94219D279795B
:1046BC00B1713979F171D91CA14217D2F9793172E2
:1046CC00B979717208301B1DA3421146DBD30499D2
:1046DC000818801C06B0F0BD04990818001D06B01F
:1046EC00F0BD04990818801D06B0F0BD0499081897
:1046FC00083006B0F0BDC0463000002024FEFFFF9D
:10470C00F0B583B03C210127484847542C2147542D
:10471C000024202110250564416407218464C464AD
:10472C0081634163082644628462C6618776048390
:10473C0039033F4A0163011D0C7702607905FA07C2
:10474C0042608460C46001614661029401940094EB
:10475C00FBF796FD002801D006F0BBFE02940194F5
:10476C00009732486946FBF7A9FF002801D006F0F4
:10477C00B0FE0294042001902E4800902B4869460C
:10478C00FBF79CFF002801D006F0A3FE02940196D3
:10479C002948009025486946FBF790FF002801D076
:1047AC0006F097FE02940C200190244800901F48BC
:1047BC006946FBF783FF002801D006F08AFE0294BD
:1047CC0001951F48009019486946FBF777FF0028B0
:1047DC0001D006F07EFE1B4D0295142001901A4864
:1047EC00009012486946FBF769FF002801D006F0DB
:1047FC0070FE029518200190144800900B486946F1
:10480C00FBF75CFF002801D006F063FE02941C202D
:10481C0001900F48009005486946FBF74FFF0028B0
:10482C0001D006F056FE03B0F0BDC046940D00203A
:10483C000024014002000004040000080800000CE1
:10484C001000001004FFFF070001002000020024EC
:04485C00000400282C
:10486000F0B58BB000240A94099408940794069438
:10487000026845498A4201D00BB0F0BD0290012385
:1048800019054248C2680A43C260C2680A400592DC
:104890000599016819430160016819400493059165
:1048A00005990168022203921143016000681040DB
:1048B0000590059808940327079706930520019013
:1048C000050706AE28463146FCF754FF08940797C3
:1048D0000398069028463146FCF74CFF089407974A
:1048E00004200090069028463146FCF743FF0894C8
:1048F00007970498069026483146FCF73BFF08943A
:1049000007970398069022483146FCF733FF089436
:104910000797009806901E483146FCF72BFF089435
:1049200007970820069028463146FCF723FF089495
:1049300007971020069028463146FCF71BFF154DBF
:104940002C621548286001986860AC60EC602020FB
:10495000049AD102120280232B616A61A961E86185
:104960002846FCF7DFFA002801D006F0B8FD0298CF
:10497000A86205650C2000210A46FCF745FA0C20C8
:10498000FCF75EFA0BB0F0BD002401403410024089
:0C49900000040050F80D00200800024058
:10499C00F0B589B007910646049008AD222003902B
:1049AC0028700520070701200190C40300220692FD
:1049BC003846214607F0ACF80A20059000900323F6
:1049CC000293304629462A46FDF70EFE384621460C
:1049DC00019E324607F09CF842202870A8780721E7
:1049EC00014007980143697038462146069A07F042
:1049FC008FF8059800900223049829462A46FDF763
:104A0C00F3FD38462146324607F082F803982870A9
:104A1C0038462146069A07F07BF8059800900498D2
:104A2C0029462A46029BFDF7DFFD384621463246D1
:104A3C0007F06EF8A87807990840884201D109B0B0
:104A4C00F0BD024804F034F8FEE7C046EEBD0008A5
:104A5C0080B53121C900415881670146CC314A8863
:104A6C007C23C252CC22825A7C30428089684160BD
:104A7C000248002102F0F2F980BDC046300000204F
:104A8C0010B504468034616D616061688022805885
:104A9C00091A7D20C20005480068504304F0D4FF79
:104AAC00A0600348002102F0D9F910BD600F00206E
:044ABC0030000020A6
:104AC00010B5CC200A4C205A8C216052605E7E21A9
:104AD000615E411A7D20C20006480068504304F020
:104AE000B9FF902160500021204602F0BDF910BDB1
:084AF00030000020680F0020D7
:104AF800F0B581B00546324805F09CF89435A868B1
:104B0800002858D0A86804F003FF2E4B002204F0B8
:104B180071FD2D4AC0CA32463B4604F06BFD2B4B53
:104B2800002206F0FAFC04F063FE2860688FA88073
:104B3800288FE880264832463B4605F07BF8A8686F
:104B480004F0E6FE00221F4B04F054FD0246214803
:104B58000B4605F06FF80420285E04F0D9FE1E4EBF
:104B68000022334604F046FD02461C480B4605F079
:104B780061F80620285E04F0CBFE0022334604F0DC
:104B880039FD024616480B4605F054F8286804F02B
:104B9800BFFE00220D4B06F0C0FC024611480B4632
:104BA80005F048F8104805F045F81048002102F0D3
:104BB80057F901B0F0BD0E4803F07CFF01B0F0BD1D
:104BC800EEBF000800408F40A005002080842E41E1
:104BD80067C1000858BD00080000594067BD0008BB
:104BE80000C0000800C400080AC000083000002007
:044BF80084C100086C
:104BFC00F0B583B03A4805F01BF8CE24394F385B3A
:104C0C00A0217852785E04F081FE374E00223346A4
:104C1C0004F0EEFC024635480B4605F009F8385F07
:104C2C009821795E3C46401A04F070FE0290019186
:104C3C000022334604F0DCFC02462D480B4604F0FF
:104C4C00F7FF2C480668436800932B48324604F063
:104C5C00EFFF9C27E05904F059FE284B002204F08A
:104C6C00C7FC024626480B4604F0E2FFE0592746F3
:104C7C0004F04CFE0022214B04F0BAFC3246009B9F
:104C8C0004F0B6FC1F4B002204F0C6FB029A019BF9
:104C9C0004F0AEFC1C4C0022234606F03CFC04F055
:104CAC00A5FDA4217850785804F030FE002223464C
:104CBC0004F09EFC00220C4B06F02DFC134B002242
:104CCC0004F0AAFB024612480B4604F0B1FF11484F
:104CDC0004F0AEFF3846002102F0C0F803B0F0BD7E
:104CEC0072BD0008300000200000594089BD00084A
:104CFC0020C000089005002098BD000800408F409F
:104D0C002EC000080000F0BF65CDCD410000F03F83
:084D1C00CBBD000814C400081F
:104D2400F0B58FB005200407012209921103079101
:104D3400204606F0F1FE9620FBF794FA77482021EE
:104D44000026324606F0E8FE9620FBF78BFA7348FD
:104D54002021099A06F0E0FE9620FBF783FA20460C
:104D64000799324606F0D8FE072002210691324602
:104D7400FCF748F80720FCF761F80DAF32460596BA
:104D8400BE7067483880099EF5032046294606F020
:104D9400C3FE0A200A900090624839463A46069BB0
:104DA400FDF726FC20462946324606F0B5FE2620AD
:104DB400387020462946059A0A9E06F0ADFE0096F4
:104DC4000323584839463A46FDF712FC2046089515
:104DD4002946099A06F0A0FEB8780A2800D099E07E
:104DE4009620FBF73FFA4F482021FFF7D5FD0DAD84
:104DF400232006902870002209922046089F3946F5
:104E040006F08AFE009603230493464829462A4660
:104E1400FDF7EEFB012205922046394606F07CFEA2
:104E2400432002902870A878EF2101406970204641
:104E34003946099E324606F06FFE0A980090022316
:104E44000393384829462A46FDF7D2FB20463946C3
:104E5400059A06F061FE06982870204639463246C7
:104E640006F05AFE0A9800902E4829462A46049EC7
:104E74003346FDF7BDFB20463946059A06F04CFE45
:104E84000DAD0698287020463946099A06F044FE6E
:104E94000A980090234829462A463346FDF7A8FB82
:104EA40020463946059E324606F036FE02982870A2
:104EB400A8789F2101402031697020463946099A1B
:104EC40006F02AFE0A980090164829462A46039BB3
:104ED400FDF78EFB20463946324606F01DFE069845
:104EE400287020463946099A06F016FE0A98009062
:104EF4000C4829462A46049BFDF77AFB204639468E
:104F0400324606F009FEA878800611D4064803F05C
:104F1400D3FDFEE7054803F0CFFDFEE70004005093
:104F2400460A0000300D002009BE000830C4000805
:104F34000DAD099EAE703420687051202870204653
:104F44003946324606F0E8FD0A98009011480223DB
:104F540029462A46FDF74CFB012206922046394693
:104F640006F0DAFD3120287020463946324606F034
:104F7400D3FD0A9800900323064829462A46FDF7E4
:104F840037FB20463946069A06F0C6FDA878342831
:104F940008D001E0300D0020014803F08DFD01E050
:104FA40038C000080DAE099AB2700D4830800BADC0
:104FB400AA702A802046394606F0AEFD0A98009071
:104FC4000848032331462A46FDF712FB01222046F6
:104FD400394606F0A1FD2878FF280CD104E0C0462C
:104FE40025EC0000300D00200DA800780BA94978AD
:104FF400814200D1A2E00DAE099AB2700C48308013
:105004000BADAA702A802046394606F085FD0A9821
:1050140000900848032331462A46FDF7E9FA0122A5
:105024002046394606F078FD2878FF280AD103E0A7
:1050340025EC0000300D00200DA800780BA949785C
:1050440081427BD00DAE099AB2700D4830800BAD11
:10505400AA702A802046394606F05EFD0A98009020
:105064000848032331462A46FDF7C2FA01222046A6
:10507400394606F051FD2878FF280BD104E0C046DC
:1050840025EC0000300D00200DA800780BA949780C
:10509400814253D00DAE099AB2700D4830800BADE9
:1050A400AA702A802046394606F036FD0A980090F8
:1050B4000848032331462A46FDF79AFA012220467E
:1050C400394606F029FD2878FF280BD104E0C046B4
:1050D40025EC0000300D00200DA800780BA94978BC
:1050E40081422BD00DAE099AB2700E4830800BADC0
:1050F400AA702A802046394606F00EFD0A980090D0
:105104000948032331462A46FDF772FA0126204650
:105114003946324606F000FD2878FF2806D000F014
:1051240000FDC04625EC0000300D00200DA80078DD
:105134000BA94978814201D000F0F3FC0BA8099A2D
:1051440081786020049001430DAE06917170452072
:10515400059030700BAD2A802046394606F0DCFC01
:105164000A9800900748022331462A46FDF740FA80
:1051740001222046394606F0CFFC2878FF280AD1C0
:1051840002E0C046300D00200DA800780BA9497834
:10519400814200D19AE00DAE069870700598307087
:1051A4000BAD099A2A802046394606F0B5FC0A98C8
:1051B40000900748022331462A46FDF719FA0122D6
:1051C4002046394606F0A8FC2878FF2808D101E0DB
:1051D400300D00200DA800780BA94978814275D0C4
:1051E4000DAE06987070059830700BAD099A2A8040
:1051F4002046394606F090FC0A980090074802239E
:1052040031462A46FDF7F4F901222046394606F0D4
:1052140083FC2878FF2809D102E0C046300D002025
:105224000DA800780BA9497881424FD00DAE06989D
:105234007070059830700BAD099A2A802046394663
:1052440006F06AFC0A9800900748022331462A4671
:10525400FDF7CEF901222046394606F05DFC287898
:10526400FF2809D102E0C046300D00200DA80078C7
:105274000BA94978814229D00DAE06987070059823
:1052840030700BAD099A2A802046394606F044FC5A
:105294000A9800900848022331462A46FDF7A8F9E7
:1052A400012620463946324606F036FC2878FF2887
:1052B40004D000F045FCC046300D00200DA8007855
:1052C4000BA94978814201D000F03AFC0DAD099F49
:1052D400AF8011480D9011480222294606F0F4FAD5
:1052E400A8700BAEB7800B97204608993A4606F093
:1052F40013FC0A9800900A48062329463246FDF713
:1053040077F901222046089906F006FC301D069024
:105314003078FF282BD105E025EC0000CC0E0020CE
:10532400300D00200DA800780BA9497881421ED1C8
:105334000DA840780BA98978814218D10DA88078EE
:105344000BA9C978814212D10BA8457903480122DF
:10535400069906F0B9FAA84209D101E0CC0E002062
:105364000BA8007904990840602800D13BE10DADF9
:10537400AF8010480D9010480222294606F0A4FA86
:10538400A8700BAEB7800B97204608993A4606F0F2
:10539400C3FB0A9800900948062329463246FDF7C4
:1053A40027F901222046089906F0B6FB3078FF2839
:1053B4002BD105E025EC0000CC0E0020300D0020A0
:1053C4000DA800780BA9497881421ED10DA8407818
:1053D4000BA98978814218D10DA880780BA9C978C6
:1053E400814212D10BA8457903480122069906F09F
:1053F4006BFAA84209D101E0CC0E00200BA8007979
:1054040004990840602800D1EDE00DADAF8010484C
:105414000D9010480222294606F056FAA8700BAEE9
:10542400B7800B97204608993A4606F075FB0A9810
:1054340000900948062329463246FDF7D9F801228F
:105444002046089906F068FB3078FF282BD105E048
:1054540025EC0000CC0E0020300D00200DA80078B3
:105464000BA9497881421ED10DA840780BA98978EF
:10547400814218D10DA880780BA9C978814212D134
:105484000BA8457903480122069906F01DFAA842A3
:1054940009D101E0CC0E00200BA800790499084042
:1054A400602800D19FE00DADAF8010480D901048EA
:1054B4000222294606F008FAA8700BAEB7800B97B3
:1054C400204608993A4606F027FB0A9800900948B6
:1054D400062329463246FDF78BF801222046089917
:1054E40006F01AFB3078FF282AD105E025EC0000ED
:1054F400CC0E0020300D00200DA800780BA94978AF
:1055040081421DD10DA840780BA98978814217D119
:105514000DA880780BA9C978814211D10BA84579CF
:1055240003480122069906F0CFF9A84208D101E008
:10553400CC0E00200BA8007904990840602852D0B2
:105544000DADAF8010480D9010480222294606F098
:10555400BBF9A8700BAEB7800B97204608993A4662
:1055640006F0DAFA0A9800900948062329463246DA
:10557400FDF73EF80125204608992A4606F0CCFAA4
:105584003078FF2806D0C1E225EC0000CC0E0020C4
:10559400300D00200DA800780BA94978814200D075
:1055A400B4E20DA840780BA98978814200D0ADE21D
:1055B4000DA880780BA9C978814200D0A6E20BA877
:1055C400467904480122069906F07EF9B04203D0D8
:1055D4009CE2C046CC0E00200BA800790499084038
:1055E400602800D092E2089F10480D9010480DAD3D
:1055F4000222294606F068F9A870099A0B922046FF
:10560400394606F089FA0A9800900A480BAE04233A
:10561400294632460693FCF7EBFF01222046394621
:1056240006F07AFA3078FF2819D105E0F2EC000090
:10563400CC0E0020300D00200DA800780BA949786D
:1056440081420CD10DA840780BA98978814206D1FA
:105654000DA880780BA9C978814200D1DBE01048FD
:105664000D9010480DAD0222294606F02DF9A870C0
:10567400099A0B922046394606F04EFA0A98009091
:1056840009480BAE042329463246FCF7B1FF012238
:105694002046394606F040FA3078FF2819D105E053
:1056A400F2EC0000CC0E0020300D00200DA8007894
:1056B4000BA9497881420CD10DA840780BA98978AF
:1056C400814206D10DA880780BA9C978814200D106
:1056D400A1E010480D9010480DAD0222294606F0B5
:1056E400F3F8A870099A0B922046394606F014FA8A
:1056F4000A98009009480BAE042329463246FCF769
:1057040077FF01222046394606F006FA3078FF2852
:1057140018D105E0F2EC0000CC0E0020300D002082
:105724000DA800780BA9497881420BD10DA84078C7
:105734000BA98978814205D10DA880780BA9C97875
:10574400814268D0FB480D90FB480DAD02222946EA
:1057540006F0BAF8A870099A0B922046394606F06A
:10576400DBF90A980090F5480BAE0423294632462B
:10577400FCF73EFF01222046394606F0CDF9307889
:10578400FF2811D10DA800780BA9497881420BD1CB
:105794000DA840780BA98978814205D10DA880789D
:1057A4000BA9C978814236D0F7480D90F5480DAD64
:1057B4000222294606F088F8A870099A0B9220461E
:1057C400394606F0A9F90A980090ED480BAE042377
:1057D40029463246FCF70CFF0125204639462A4665
:1057E40006F09AF93078FF2800D0B2E10DA80078CD
:1057F4000BA94978814200D0ABE10DA840780BA9F0
:105804008978814200D0A4E10DA880780BA9C978D9
:10581400814200D09DE10DAD099FAF80DB480D9022
:10582400D8480222294606F04FF8A8700BAEB7807C
:105834000B97204608993A4606F06EF90A980090AC
:10584400CF48062329463246FCF7D2FE01252046DE
:1058540008992A4606F060F9301D05903078FF2833
:1058640024D10DA800780BA9497881421ED10DA836
:1058740040780BA98978814218D10DA880780BA9AA
:10588400C978814212D10BAE7779BE4805992A4670
:1058940006F01AF8C01B411E88410699715600296A
:1058A40000DA00252843012800D05EE10DAD099FF0
:1058B400AF80B6480D90B3480222294606F004F89A
:1058C400A8700BAEB7800B97204608993A4606F0AD
:1058D40023F90A980090AA48062329463246FCF781
:1058E40087FE0125204608992A4606F015F93078E6
:1058F400FF2824D10DA800780BA9497881421ED134
:105904000DA840780BA98978814218D10DA8807818
:105914000BA9C978814212D10BAE777999480599C0
:105924002A4605F0D1FFC01B411E884106997156D5
:10593400002900DA00252843012800D015E10DAD27
:10594400099FAF8091480D908E480222294605F0A8
:10595400BBFFA8700BAEB7800B97204608993A4658
:1059640006F0DAF80A98009085480623294632465C
:10597400FCF73EFE0125204608992A4606F0CCF89D
:105984003078FF2824D10DA800780BA949788142EA
:105994001ED10DA840780BA98978814218D10DA891
:1059A40080780BA9C978814212D10BAE77797548FA
:1059B40005992A4605F088FFC01B411E88410699B7
:1059C4007156002900DA00252843012800D0CCE0D4
:1059D4000DAD099FAF806D480D906A48022229469B
:1059E40005F072FFA8700BAEB7800B97204608999C
:1059F4003A4606F091F80A98009061480623294631
:105A04003246FCF7F5FD0125204608992A4606F0A2
:105A140083F83078FF2824D10DA800780BA94978A1
:105A240081421ED10DA840780BA98978814218D1F2
:105A34000DA880780BA9C978814212D10BAE777971
:105A4400504805992A4605F03FFFC01B411E884176
:105A540006997156002900DA00252843012800D050
:105A640083E00DAD099FAF8048480D904548022260
:105A7400294605F029FFA8700BAEB7800B97204686
:105A840008993A4606F048F80A9800903C480623DC
:105A940029463246FCF7ACFD0125204608992A46E2
:105AA40006F03AF83078FF2824D10DA800780BA925
:105AB400497881421ED10DA840780BA9897881428A
:105AC40018D10DA880780BA9C978814212D10BAEE8
:105AD40077792C4805992A4605F0F6FEC01B411E2D
:105AE4008841069971560029294600DA0999084324
:105AF40001283AD1ED024B2086006436204629461F
:105B040006F012F83046FAF7ADFBF7E7ED024B204A
:105B140086002046294606F007F83046FAF7A2FB2D
:105B2400F7E7F5022046294605F0FEFFC820FAF7FC
:105B340099FBF7E7F2EC0000CC0E0020300D0020BA
:105B4400F5022046294605F0EFFFFA20FAF78AFB12
:105B5400F7E7ED024B20860032362046294605F051
:105B6400E3FF3046FAF77EFBF7E79620FAF77AFB75
:105B740001222046079905F0CFFF0FB0F0BDC046C3
:105B8400300D0020CC0E0020F2EC000021EC0000CF
:105B9400F0B58BB008AE0025357209959948089088
:105BA40099480222314605F08FFEB07005AF3D7270
:105BB400069505950520000703900124E10304914F
:105BC4000295002205F0A8FF0A2000908F480923BF
:105BD40031463A46FCF70CFD0398049903940122DC
:105BE40005F09AFF3878FF282DD108A8007805A978
:105BF4004978814227D108A8407805A9897881424B
:105C040021D108A8807805A9C97881421BD105A8AB
:105C1400047A011D7C48042205F056FEA04212D1EC
:105C240005A80079CC21014084290CD105A841792B
:105C34000904827912025218C0791318C80D0BD0C6
:105C440074481B1808E0C120400071490A5A521CCC
:105C54000A52FFF765F82B466F4908686F4A90426D
:105C640007D0421C0A60132801DC002000E0012058
:105C740003906B480068C118C20F801840100E1AB8
:105C8400F00F301847103120C000614B1F50986F3F
:105C940002901C46C834E068049480215958882234
:105CA4009A58401A504303F035FE5E4B002203F02D
:105CB400A3FC03F09FFD63218900554B58505849BC
:105CC4000E600299791A584A1160091A02915748CC
:105CD40001600420205E7E21595E1E46401A03F0B6
:105CE40019FE04460F469020305803F013FE224656
:105CF4003B4605F014FC00224A4B03F07DFC03F004
:105D040079FD0299081A4A49086003F003FE494BD9
:105D1400002205F004FC484B002205F000FC7D2223
:105D2400D305002205F0FBFB06460F4643480660F8
:105D340041609420364C205803F0ECFD404B002287
:105D440003F05AFC32463B4605F0E9FB02900F464D
:105D54003C4981C106200499085E9821615E401A7D
:105D640003F0D8FD04460E46A4202949085803F040
:105D7400D1FD354B002203F03FFC2246334605F0AB
:105D8400CEFB324B002203F04BFB029A3B4605F05C
:105D9400C6FB06460F462E48066041602D4B304632
:105DA400002203F0E7FC002811D100222A4B3046E0
:105DB400394603F0FFFC002809D10022194B304674
:105DC400394605F0ACFB03F015FD114A03E0192038
:105DD40000010F4A1058E421505003980028049AF7
:105DE4000BD0D069116A884201DDD0691062D06994
:105DF400516A884201DAD069506218480121016071
:105E04000BB0F0BD12EC0000CC0E0020300D0020D1
:105E140030000020010000FFAC0F0020FFFFFF7FD7
:105E2400B00F002000408F40600F0020680F00205A
:105E3400640F00200000084000004940A005002035
:105E440080842E419005002065CDCD410000F03FB7
:105E54009805002000206140002061C0400F002010
:105E64000548C16D054A4A4305218901425040183D
:105E7400D11741607047C04630000020F0F1FFFFA9
:105E8400F0B589B0DC4DE86DE1210B01010C1C0C6F
:105E9400002208939BB2594380B202934343039474
:105EA4000C0C090459185441002200204018069093
:105EB40062410792D14B03CB083B014307D1002039
:105EC4004B2189006958CE4A4A431A605860CD4B29
:105ED40003CB083B014307D1002013210901695872
:105EE400C74A4A431A605860E42428590028059494
:105EF4000FD45220285A03F049FD0022C24B03F06C
:105F04007BFB06460F46285903F004FD32463B4608
:105F140030E0E86D6821695A03F0C2FD064628594D
:105F240071428842285929DA03F0F4FC04460F46EA
:105F34000491304603F0EEFC02460B460120C107F3
:105F44007940204603F058FB01900F465020285A10
:105F540003F01CFD0022AC4B03F04EFBAB4B0022C4
:105F640003F05EFA02460B460198394603F0ECF85A
:105F74002246049B05F0D3FA03F03CFC2C46C834BB
:105F8400A0627020285EA16A081AA062E169E06933
:105F9400002912D4C1179B4D2A6816186F684F4107
:105FA400974A00233046394603F0B6FD1321090110
:105FB400914A5050C0C5904D1BE04042C1178F4BD1
:105FC4001A6816185F684F418D4A002330463946D7
:105FD40003F0A2FD4B218900685069587D20C00060
:105FE4004843E96D03F05CFD4F2189006852834802
:105FF400C0C0A06A616BC217236B181820634A41A2
:106004006263A06AE16FC217A36F1818A0674A41C0
:10601400E267A06FE16F0026089A334603F064FD3F
:106024002D21C90004916850606B216B069A511AA6
:106034000799814105DAF8202A502846F830079953
:1060440041600520800129184A682B585B1EB24123
:1060540001DB2E504E60E96D5420285AD827EA59A6
:106064005823EB5A9A4211DD484303F08FFC664BE8
:10607400324603F0C1FA03F0D7FB059AAA58D317A6
:10608400101A8B4102DA62480088461C6048068078
:106094005620285A31B281420BDD07986063069876
:1060A40020630020E067A06702F0D6FC5948012174
:1060B4000160206B616B0026089A334603F014FDDF
:1060C400E06220690321C901695A88422FDAE8593C
:1060D4007D21C90088422ADD4F480188491C01807E
:1060E40089B20A2925D34B4C2168012921D10A21DF
:1060F40001800920400129580909E12913D32858AE
:10610400464988420FD8049968580028685800D531
:10611400404243218900685002F0BCFB0021216009
:10612400284600F09FFE492080002E5001E03A48A6
:1061340006806420285A042830D8C0467844007960
:1061440040008744023025282200E86D0023010C1A
:10615400039C22464A43029E714380B246436043F5
:106164000F0C090471185741040C000446187C41B3
:10617400F82028582946F8314968294A03F050FC88
:106184003246234603F0B0FC07E002F01FFC04E0B3
:1061940002F0BAFB01E002F0E1FB06460120000236
:1061A4002E5009B0F0BD04996858002801D400208D
:1061B40001E068584042432189006A58002A02DD00
:1061C4006F58F91701E0EF6D00210891C117144EC3
:1061D40000243246234603F023FC3A46089B03F08E
:1061E40083FC721E2346A341121A8B4100DB341A2E
:1061F4000029D3D42646D1E730000020B80500207A
:1062040080EE3600C0050020000059400000F0BFB9
:10621400B80F00203C0F0020B60F002080FC0A00BD
:04622400A08601004F
:10622800F0B583B035490B68354A934206D05A1CFD
:106238000A6034498B4201DC002100E00121019110
:10624800314B19680A0A891A029009181960080A54
:10625800304E718800250A0C070C3B46534380B228
:1062680042438CB260437C43170C110440185F41D1
:10627800210C22041018794106222B4603F0CEFB8C
:1062880003F090FB224B002203F0B4F903F0B0FABC
:106298003061019800280BD030697169884201DDAE
:1062A800306970613069B169884201DA3069B0617A
:1062B800CA20164E305A029C210C020C13464B433E
:1062C80080B24143A4B2604354430A0C0904401805
:1062D8005A41210C2304181851410622002303F0C7
:1062E8009DFB03F05FFB0A4B002203F083F903F0E8
:1062F8007FFA65218900705003B0F0BDA40F00201B
:10630800FFFFFF7FFF090000A80F002030000020DA
:0863180000002441F800002000
:1063200010B582B00848026801210A430260006883
:1063300008400190019809200022FAF765FD092024
:0C634000FAF77EFD02B010BD38100240DC
:10634C0010B5104909680906890B0F4A895C0028A9
:10635C0000D0017038290DD0FF2906D039290ED173
:10636C000C4802F0A5FB012010BD084802F0A0FB70
:10637C00002010BD064802F09BFB022010BD03203C
:10638C0010BDC046E075FF1F00F8FF0756C000089F
:08639C0024BE0008DDC1000869
:1063A400F0B583B00090554802F086FB544E0125A9
:1063B400358428044B210902B161F06130462A304A
:1063C4001E2104F069FDB8204E493150B4204E49D5
:1063D4003150B0204D493150AC204D4A3250A820A4
:1063E4003150A4203250A2207D2101913152C72086
:1063F400C0434B30A02170529C2046493150982014
:106404004549315096200227375294203554AF2005
:10641400800170309221705290204049315288207E
:106424003F49315080203F493150304618303E4971
:1064340041673E49C1663E4900203E4AB264F06469
:1064440030657065B165BC217050D0217050CC218D
:106454005A2272523146BC3148608860C860C143D8
:10646400354CFB43354A30667066B166F166326777
:106474007167B467F367D820706039203070B068F2
:10648400401CB060FAF7CCFF0198C000FAF76EFF29
:106494002B480168C90702D00168A9430160294853
:1064A4000760294C21680906490E491E8160C560B0
:1064B40002A9FBF75DF8002800D0FEE7206800067B
:1064C400800B224FC519FF2084020CCE01202946DF
:1064D400083EFAF773FE0028FED11B4800688002CC
:1064E40020403818D430083608358542EDD3FAF701
:1064F400ABFF009800F02CF803B0F0BD0AC200080E
:10650400E803002010270700320038FF54F248F453
:106514004C1D581B60EAC0DAC02BE02EB0360000D8
:1065240080482800630069000A000200A086010078
:1065340040420F0090D00300007884C900D68AEA54
:10654400142002402C0F0020E075FF1F00F8FF0705
:10655400F0B59CB04321890041180291CA490968E9
:1065640009068A0BC9495618711C1B91B11C1A9152
:10657400F11C1991311D1891711D1791B11D1691BE
:10658400F11D1591314608311491314609311391A9
:1065940031460A31129131460B31119131460C3199
:1065A400109131460D310F9131460E310E91314625
:1065B4000F310D91314610310C91314611310B914F
:1065C400314612310A913146133109913146143161
:1065D40008913146153107913146163106913146FD
:1065E4001731059131461831049137461937314630
:1065F4001A31D723DC4302464032009203908C3098
:106604000190A34805193019D823C05CE8541B989D
:106614000019C05CD922A8541A980019C05CDA2267
:10662400A85419980019C05CDB22A85418980019C2
:10663400C05CDC22A85417980019C05CDD22A85461
:1066440016980019C05CDE22A85415980019C05C85
:10665400DF22A85414980019C05CE022A8541398AF
:106664000019C05CE122A85412980019C05CE2220F
:10667400A85411980019C05CE322A854109800197A
:10668400C05CE422A8540F980019C05CE522A85409
:106694000E980019C05CE622A8540D980019C05C3D
:1066A400E722A8540C980019C05CE822A8540B985F
:1066B4000019C05CE922A8540A980019C05CEA22B7
:1066C400A85409980019C05CEB22A8540898001932
:1066D400C05CEC22A85407980019C05CED22A854B1
:1066E40006980019C05CEE22A85405980019C05CF5
:1066F400EF22A85404980019C05CF022A854381959
:10670400C05CF122A8540819C05CF222A8541B34BE
:1067140000D076E75E4CA06903990861A08B88825B
:10672400E08BC882208C0883608C8883A08CC8830B
:10673400E08C0884208D4884608D009EB087A08DF5
:10674400F087E08D019DA881208EE881608E2880ED
:10675400A08EA882E08EA883A06B3064E06B706486
:10676400206CB064606C6860A06C2861E06CA86107
:10677400206D2862606D8867A06DA8608020205A13
:1067840070828220205A308220461830C06EC8653C
:106794008820205808668C20205AB0828E20205AE7
:1067A400F0829020205A30839220205A70839420C3
:1067B400205CB0849620205A30859820205A888600
:1067C4009A20205AC8869C20205A08879E20205A46
:1067D4004887A020205A8887A220205AC887A4204E
:1067E400205A3080A620205A7080A820205AB080D9
:1067F400AA20205AF080AC20205A3081AE20205AA2
:106804007081B020205AB081B220205AF081B42087
:10681400205A7085B620205AB085B820205AF085B9
:10682400BA20205A3086BC202058029A1062C02018
:1068340020585062C42020589062C8202058D0624A
:10684400CC20205A7086D0202058D061206EE86673
:10685400606E2867A06E1060E06E5060606F906399
:10686400206F5063E06F1064A06FD063E0684860ED
:10687400207839214140A2885A40E08810430843D7
:10688400411E88411CB0F0BDE075FF1F00F8FF07F2
:04689400E8030020F5
:10689800F0B59FB004910090E24802F00BF9E2488D
:1068A80000680006800BE1494218901C1D90D01C1E
:1068B8001C90101D1B90501D1A90901D1990D01DF2
:1068C8001890104608301790104609301690104658
:1068D8000A30159010460B30149010460C30139067
:1068E80010460D30129010460E30119010460F30A1
:1068F8001090104610300F90104611300E90104630
:1069080012300D90104613300C90104614300B9036
:10691800104615300A901046163009901046173068
:106928000890104618300790104619300690501CF1
:106938000590FF218902029100210391C943019129
:10694800CF39BB4E374676185518D023ED5CF55431
:1069580005984518ED5CD12435551D984418E45C1C
:10696800D22574551C984418E45CD32574551B989B
:106978004418E45CD42574551A984418E45CD52569
:10698800745519984418E45CD62574551898441819
:10699800E45CD725745517984418E45CD82034541F
:1069A800169C6418E45CD9257455159C6418E45C3D
:1069B800DA257455149C6418E45CDB257455139C23
:1069C8006418E45CDC257455129C6418E45CDD25CD
:1069D8007455119C6418E45CDE257455109C641889
:1069E800E45CDF2574550F9C6418E45CE02574555D
:1069F8000E9C6418E45CE12574550D9C6418E45CF5
:106A0800E22574550C9C6418E45CE32574550B9CD2
:106A18006418E45CE42574550A9C6418E45CE52574
:106A28007455099C6418E45CE6257455089C641840
:106A3800E45CE7257455079C6418E45CE825745504
:106A4800069C6418E45CE92574553E461A3100D06A
:106A580078E71B90706DF24C6065708D6085B08D25
:106A6800A085706B1A90B16BF26B306C1D90756CD1
:106A7800B06C1C90F06C1990306D1890708E608618
:106A8800B06DA065F08DE085308E20861A98606321
:106A9800A163E2631D98206465641C98A06419983A
:106AA800E06418982065049D012D04D0B069A061A8
:106AB800039805D105E04B200002A061039800E08F
:106AC800B08BA083012D03D1E58304D1632004E0BA
:106AD800F08BE083FAD07820305A328C80216052D3
:106AE800012D01D0705800E0CE4888211A916050DD
:106AF800012D02D08420345A00E00A248C21C84891
:106B08001C914452012D02D07A24345B00E06924A0
:106B1800822544530446049D012D0ED02284039AF5
:106B28000ED16284012D039A0FD1A284039AE284C4
:106B3800039A228517E0F26F16E02584039AF0D0B5
:106B4800728C6284012D039AEFD0B28CA284012D3D
:106B5800039AECD0F28CE284012D039AE9D0328DAD
:106B68002285012DE7D1B04A1834E2660222012DB0
:106B78001D9201D08622B25A8E20A94C1990225219
:106B8800012D02D01A98315A00E0A84990201A9095
:106B98002152AF218901012D03D08A24355BA04CF5
:106BA80001E00D4670359226A553049C012C01D1B5
:106BB800204601E01C98385C9425994A5055012CD0
:106BC8001D9C01D019983C5A96201452049C012C03
:106BD80001D01A99795A9822914C1A92A152049983
:106BE800012901D0BC5B00E0914C3E469A228C49B9
:106BF80019928C52049C012C01D0745B00E08D4CDE
:106C08009C268C53049D012D01D0385A00E08A48F7
:106C18009E240853C720C043012D1C900AD01A98FF
:106C2800385A08E06BBE0008E075FF1F00F8FF0740
:106C3800C00400204B30A02288527D20012D1A90DC
:106C480001D01998385AA222189288527B48012DEF
:106C580000D0B85BA422724917928852385B784AF0
:106C6800012D00D00246A8216D4C19916252754C35
:106C7800012D224600D00246A620694E3252724AA1
:106C8800012D164601D018997E5AAA2564491895EF
:106C98004E53049E012E694D01D017997D5AAC269A
:106CA8005F498D53049D012D00D03C5AAE255C48A8
:106CB800445304980128624901D01998395AB024DC
:106CC800574801530498012801D018983A5AB2201D
:106CD80053490A520499012901D0BA5B00E03222D3
:106CE800B4214F4E7252049A012A01D07A5B1C9249
:106CF800B6224B4D1C9EAE52049D012D01D03C5B2B
:106D080000E0524CB822464EB452012D01D0385AF8
:106D180000E00720BA2430533446012D039800D0F0
:106D28007858BC216050012D039800D0B858C02174
:106D38003B4C6050C420012D01D0395A00E05A2143
:106D4800CC22A152C821012D039A00D07A58E250D2
:106D5800039B635023501D98C0433D493D4A236619
:106D68006366019CB466F46632672D4A54672C4CFE
:106D7800A167E067B868401CB8601B996160A060B3
:106D880039202070012D184600D0387C2074012D40
:106D9800224E01D0F86803900398E060FAF73EFBB2
:106DA8001A98C000FAF7E0FA2B480168C90703D01F
:106DB8000168012291430160284802210160164FB1
:106DC800396801220906490E491E8160C2601EA960
:106DD800FAF7CCFB002800D0FEE738688002029959
:106DE800084085190CCC01202946083CFAF7E4F93B
:106DF8000028FED138688002029908403018D43043
:106E0800083408358542EDD3FAF71CFB0098FFF7E4
:106E18009DFB1FB0F0BDC046E075FF1F00F8FF07DF
:106E2800E803002080482800A0860100B036000052
:106E3800E02E000060EAFFFFC0DAFFFF4C1D0000F3
:106E480054F2FFFF581B000048F4FFFF1027000012
:106E5800007884C900D68AEA142002402C0F00204A
:106E6800F0B583B001910446804801F023FE206903
:106E78007F4EB061A08AB083E08AF083208B308493
:106E8800A08B7084E08BB084208CF084608C30857B
:106E980021464031C88FB085888F708520468C3058
:106EA8008289F285C28932868C22A35A7386838AA4
:106EB800B386838BF3860B6CB3634B6CF3638B6C79
:106EC8003364436873640369B3648369F364036A6E
:106ED8003365A36F73658368B3654B8A8027F35363
:106EE8000B8A8227F353E36D37461837FB66236E08
:106EF8008827F3518B8AB352CA8A8E23F2520A8B9F
:106F08009023F2524A8B9223F2528A8C9423F254A1
:106F18000A8D9623F252A28E9823F252E28E9A2379
:106F2800F252228F9C23F252628F9E23F252A28F3A
:106F3800A023F252E28FA223F2524022A25AA423A3
:106F4800F2524A88A623F2528A88A823F252CA88A3
:106F5800AA23F2520A89AC23F2524A89AE23F2528A
:106F68008A89B023F252CA89B223F2524A8DB423D5
:106F7800F2528A8DB623F252CA8DB823F2520A8E83
:106F8800BA23F25243229300E218176ABC257751BC
:106F9800556AC027F551956AC427F551D56AC8279F
:106FA800F551498ECC257153D169D0257151016FA6
:106FB8007166C06E3066E058B0665068F066506B17
:106FC8003067906B7067D06BB067106CF0673920D2
:106FD8003070D8207060B068401CB06001980028FC
:106FE80004D0244801F066FD6068F060FAF716FAEC
:106FF8007D20C000FAF7B8F91F480168C90703D017
:1070080001680122914301601C48022101601C4D66
:10701800296801220906490E491E8160C26002A939
:10702800FAF7A4FA002800D0FEE728680006800BCB
:1070380014494518FF2087020CCE01202946083E36
:10704800FAF7BAF80028FED10D48006880023840E7
:107058000C490818D430083608358542ECD3FAF7BD
:10706800F1F92046FFF772FA03B0F0BD1FC200081D
:10707800E803002054C40008142002402C0F00200C
:08708800E075FF1F00F8FF078F
:1070900070B54F2080000F4E305A002816D0C836E9
:1070A000F06E02F075FC04460D46306F02F070FC85
:1070B00002460B462046294602F0A0FA0022074B62
:1070C00004F02FFA02F098FB00B270BD024800B243
:1070D00070BDC04630000020FFFF00000000594096
:1070E000F0B585B08A4800688A4A1446C834216ED3
:1070F000081ACD2149005052874D281D7C2629466B
:10710000324603F0D5FE854F381D394602967C2263
:1071100003F0CEFEE069039028602069386000200B
:107120007F4B05460246194606E0001D80283B4677
:10713000049D2246314619D0784C2458E6177440F5
:10714000A71BAF423C4600DC2C4604949F42724C85
:1071500000DB1F462358DC1763401E1B9642344653
:1071600000DC14468E42E0DB0E46DEE7A01BC117B2
:107170004840451A6749C86D6824095B02F092FCD3
:10718000142102F067FC854205DA0120C043401C4F
:1071900000B205B0F0BD0498C01BC1174840401AAA
:1071A000192803D25F4800B205B0F0BD04950194E0
:1071B0005E490022D643374601E01031521C0B468F
:1071C0000C3B1D68039BEB1ADC1763401C1BBC4285
:1071D000134600DC33460E46083E3668BC4200DCEF
:1071E0003C46751BEF177D40ED1BA54200D9531C93
:1071F000A54200DC25460C1F2768BC1BE61774401F
:10720000A41BAC4200D9931CD21C1F2A10D0AC4244
:1072100000DC2C460D680395ED1BEE177540AF1B87
:10722000A742164600D81E46A742C6DC2746C4E73A
:10723000102B69D102F070FB04460D46049802F051
:107240006BFB02460B462046294602F0D7F9002484
:10725000354B224604F065F902F0CEFA472103913E
:1072600089002C4A50522520C00010582849086037
:1072700020460094049428490958A3001E46029A07
:1072800056403724E400234F3C19A15123490958A3
:10729000039AD5007D19A95178265E401E490F1822
:1072A0007968A1511D4909184A68AA5174225A40A7
:1072B000BE68A6508E68AE5070225A40FE68A65036
:1072C000CE68AE506C225A403E69A6500E69AE5050
:1072D0001A46019E72407E69A6504E69AE506422E5
:1072E0005A40BE69A6508E69AE5060225A40FB6972
:1072F000A350C969A950049C203008348028B9D112
:10730000009800B205B0F0BD002005B0F0BDC04649
:10731000980F002030000020B00C0020B00B00209F
:10732000FFFFFF7FFEFF000000408F40C00C0020E9
:10733000F0B585B08B4800688B4A1446C834216E7E
:10734000081ACD2149005052884E301D7C27314605
:107350003A4603F0ADFD864D281D294602977C2252
:1073600003F0A6FD192000017F4908580390306002
:10737000E068286000207F4B05460246194606E07B
:10738000001D80283B46049D2246314619D0784C8A
:107390002458E6177440A71BAF423C4600DC2C463D
:1073A00004949F42714C00DB1F462358DC17634056
:1073B0001E1B9642344600DC14468E42E0DB0E462D
:1073C000DEE7A01BC1174840451A6749C86D68240D
:1073D000095B02F067FBC117890F401880108542D6
:1073E00005DA0120C043401C00B205B0F0BD04988E
:1073F000C01BC1174840401A642803D25E4800B23F
:1074000005B0F0BD049501945D490022D64337468E
:1074100001E01031521C0B460C3B1D68039BEB1A1C
:10742000DC1763401C1BBC42134600DC33460E468F
:10743000083E3668BC4200DC3C46751BEF177D40B9
:10744000ED1BA54200D9531CA54200DC25460C1FAC
:107450002768BC1BE6177440A41BAC4200D9931CE0
:10746000D21C1F2A10D0AC4200DC2C460D680395BC
:10747000ED1BEE177540AF1BA742164600D81E46FF
:10748000A742C6DC2746C4E7102B68D102F044FAB5
:1074900004460D46049802F03FFA02460B46204689
:1074A000294602F0ABF80024344B224604F039F8A8
:1074B00002F0A2F98F2149002B4A50522520C0002A
:1074C000105828490860204603940494274F3C58DC
:1074D00004998A00154602994D405723DB00224942
:1074E000CB185C51224C26586724E4000C196651D5
:1074F000782656403D186F689F511D490F187968CE
:10750000A15174215140AE685E50BE686650702132
:107510005140EE685E50FE6866506C2151402E6905
:107520005E503E6966501146019E71406E695E5024
:107530007E69665064215140AE695E50BE696650F6
:1075400060215140EA695A50FA696250049C203027
:1075500008348028B9D1039800B205B0F0BD0020EE
:1075600005B0F0BD940F002030000020300C00204A
:10757000300B0020FFFFFF7FFEFF000000408F4028
:04758000400C00209B
:1075840070B5134A1368134CA34201D05B1C1360FB
:10759400401A02F0BFF904460D46CA200E4E305A76
:1075A40002F0F4F922462B4603F0B9FF00220B4BFC
:1075B40002F022F80A4B002202F01EF8094A0A4B94
:1075C40002F01AF802F016F919210901705070BD81
:1075D400900F0020FFFFFF7F30000020ECFF2341CD
:0C75E40000004440FCA9F1D24D62403F81
:1075F000F0B589B000240894079406940594049487
:107600003048016802221143016001681140039172
:10761000039901680422114301600168114003913C
:107620000399016820220292114301600168114010
:1076300003910399016801252943016000682840EE
:1076400003900398052000070090F9214E01314670
:10765000224604F063FA290201911B48224604F0F5
:107660005DFA06952120000405906802049004AF9D
:1076700015483946FAF77EF807940694059504965E
:1076800000983946FAF776F806950594402004905C
:107690000E483946FAF76EF8079406940595019856
:1076A0000490094E30463946FAF764F80794069577
:1076B00005950298049030463946FAF75BF809B010
:1076C000F0BDC046341002400004005000080050D5
:1076D00001214A02904201D1014801607047C04631
:0476E000400F002037
:1076E400A8B00027219720971F971E971D971C97D6
:1076F4001B971BA8FAF714F81F98AA2807D0CC28C0
:1077040003D0BB2806D1F64802E0F64800E0F6486C
:1077140001F0D2F9F8F75AFD1BAE3421304603F0DC
:10772400BBFB1A97199718971797169715971497DD
:1077340013971297119710970124A0020690FAF755
:107744000BF9FAF7F5F8ED4A506A18210143516232
:10775400FAF7F8F86007279060042690082025902F
:107764002497022523952295402020901F972102DB
:107774001E911D94062003901B9030460E46FAF786
:107784002DF91A971997189507200490179017A8A0
:107794000221FAF745FB05961696A0071590119756
:1077A400D748109010A8FAF793FCD64801F084F952
:1077B400FCF7B0F9FCF7B8F9FCF76AF8FFF716FF25
:1077C400FEF7ACFD00F004FEFCF79EFF00F0D6FCD3
:1077D4002103CA4D286808432860CB4809940462F1
:1077E400FF221023049C8460C360026147618761A7
:1077F40002328280C54A02602A680A401B921B99A1
:10780400F9F752FB00F098FE00F05CFFFEF728FB4E
:1078140010AC2046FEF798FDBD4948802278CA8105
:10782400032811D8784400794000874401050901F0
:10783400B748FEF7B5FD07E0B548FEF789FE03E05B
:10784400B3480021FFF726F8B24801F035F9B048F3
:10785400FEF77EFEB048402103F092FC00280FD1D1
:107864003220F8F7FFFC4021AB4803F089FC0028E4
:1078740006D1AA4801F020F9A5480121FFF70AF82A
:10788400A34E3169B28AF38AA5480090A54804F052
:107894006FF9A54C2046F9F75FF8A4490822204661
:1078A400F8F7B6FE6420F8F7DDFCFDF739FAA048D6
:1078B40001F002F900F0E0FA052002900507308B90
:1078C40000281CD00998C4020E940F970122284660
:1078D400214604F021F93746059E5E363046F8F716
:1078E400C1FC00222846214604F016F930463E46E3
:1078F4000F9FF8F7B7FC7F1C308B8742E5D3002736
:107904003046C83007900F970C970A97EE4C0B95AA
:1079140003E084202221EB4A1150ED48006801283D
:1079240020D10024EA480460E84DA86800F004FC73
:10793400286800F033FD6868FEF774FCE86829697C
:10794400FFF71EFE079D2A69D317E869C11702F0E5
:1079540067F87D22D2000023DB4C02F0C5F82864CE
:10796400FFF7E4FCDB480068012806D104F024F9A1
:10797400FFF7B4FB0020D7490860F8F76DFC014617
:10798400D5480068056840680E91CE1B701E86417C
:107994000F980028099A00DC00220F2005400C985B
:1079A4008542C64F0D9200D183E008962520C4007D
:1079B4003859401C38510A98002808D10B98069968
:1079C40004F0B2F801200102C44804F0ADF8FEF757
:1079D40057FA00F087FE00F057FA00F001FB38591F
:1079E400BF4902F05DF8BF490968884205D0BD4926
:1079F400086000213846FFF735FA6720840000F05C
:107A040017FC38538B204400FFF740FB3853AF4C2E
:107A1400E06900F099FC6069CA27A849C95B020CB7
:107A24000B0C1C46544389B24A4380B24143584329
:107A3400130C12048A186341010C00048018594184
:107A44000B22002301F0ECFF01F0AEFF0022A64B55
:107A540001F0D2FD01F0CEFE15210901974A5052E2
:107A64009A4880699549C95B020C0B0C1F46574321
:107A740089B24A4380B241435843130C12048A1812
:107A84007B418E4F010C0004801859410B220023C6
:107A940001F0C6FF01F088FF0022934B01F0ACFD1A
:107AA40001F0A8FEA921490078520C95864C089E45
:107AB4000D9A2620205C798B00290B9D00D1B8E01B
:107AC400002800D0B5E0788B8849884232DC401E1B
:107AD4000A2800D99BE005A1085C40008744C04601
:107AE400C7BE0008ACBE0008E2BE00080C4D5955E4
:107AF40097E4515E4A434700002130E038100240C9
:107B0400014002006CC00008CC0E0020003002408E
:107B1400300000208ABE00080008005099BE00080A
:107B2400A40A0020C8050020940D0020F00E0020B7
:107B340034C200086E49884209DC6F49884231D05A
:107B44006B49884263D1012000F0ECF86EE0FD211E
:107B5400890088422AD06749884258D10121384691
:107B6400FFF780F962E03846FCF7C4FF5EE0FDF7FA
:107B740043F85BE0FCF7A2FF58E03846FEF710FC40
:107B840054E03846FCF768FF50E03846FEF7E0FC66
:107B94004CE001213846FEF77DFE47E03846FCF70D
:107BA40073FF43E0002000F0BDF83FE00020219087
:107BB40020901F901E901D901C901B901BA8F9F7FD
:107BC400AFFD029800062190049800062090BB2087
:107BD4001F9003981B90F9F723FC002802D0474814
:107BE40000F06AFFF9F770FC002802D0444800F066
:107BF40063FF444800F060FF1BA8F9F71DFD00284F
:107C040007D0414800F058FFF9F772FC0EE04448F1
:107C14000AE0F9F76DFC3D4800F04EFFF9F714FC5B
:107C24003B4800F049FF3B4800F046FF00207883C2
:107C34000D9A32400F9FBF1A4021214803F0A0FA49
:107C440000280CD1002F0AD10A20F8F70BFB4021A1
:107C54001B4803F095FA002803D00F970FE00F9705
:107C64000DE00599F4310A9800280F9101D00A9784
:107C740005E00122284606990A9203F04DFF2046AA
:107C840003F098FF00280E9F00D146E62046FCF73B
:107C940025FA022800D03CE60A98002800D03CE6E9
:107CA4002046FCF715FB38E6BFF34F8F1A481B49F3
:107CB4000160BFF34F8F00BFFDE7C04630000020D6
:107CC40000080050A40A0020C8050020F00E00207F
:107CD400440F0020400F0020A00E0020000400509C
:107CE40080510100700F002000002441F1030000C6
:107CF400F3030000D2040000F2030000FDBE0008FC
:107D04008CC00008ACC40008B5C20008BCC400089C
:107D1400A2C00008D4C400080CED00E00400FA0579
:047D240060C400082F
:107D280030B587B00546002406940594049403945E
:107D38000294019400946846F9F7F0FC002D27D0CE
:107D4800444800F0B7FE0498AA2832D1BB2004901A
:107D580002200090F9F762FB002802D0344800F0B6
:107D6800A9FEF9F7AFFB002802D0334800F0A2FEC5
:107D78003A4800F09FFE6846F9F75CFC00281AD0E4
:107D8800374800F097FEF9F7B1FB002007B030BD87
:107D98000498BB281CD1AA20049002200090F9F76F
:107DA8003DFB002817D0224800F084FE002007B0D1
:107DB80030BD29480AE0F9F799FB234800F07AFE1C
:107DC800F9F740FB214800F075FE264800F072FEE6
:107DD800012007B030BD174800F06CFEF9F772FBC0
:107DE800002805D0144800F065FE002007B030BD1B
:107DF800124800F05FFE6846F9F71CFC002807D01F
:107E0800F9F774FB0E4800F055FE002007B030BDAE
:107E18000C4800F04FFEF9F769FB0B4800F04AFEEA
:107E2800F9F710FB094800F045FE0948CEE7C046BF
:107E3800FDBE00087AC000088CC0000841C20008D6
:107E480077C2000870C40008BCC40008A2C00008BB
:107E580056C200088CC4000898C20008ACC40008C8
:087E6800B5C20008D4C40008F3
:0C7E70000148012101607047440F002010
:107E7C0002480021C943C18781877047F800002060
:107E8C00F0B583B074244B4D285B002804D0285BDC
:107E9C0001281BD101221BE04748008800284748D5
:107EAC0002D083214900685283214E00A95B00292E
:107EBC0002D0A95B81424DD1D8202858A98E012728
:107ECC00884202960FDA3E483E4638E0285B002294
:107EDC00052000070121490203F01AFE285B3649F0
:107EEC00088003B0F0BDE42028583C21695E7D2257
:107EFC00D2004A43904202DA022632481FE0CE21D9
:107F0C006A5E48202B5E9A4202DD03262E4816E05C
:107F1C000197CC22AB5E285E83422C4801DD0426FF
:107F2C000DE06B5E4C216F5EBB4202DA05262848E1
:107F3C0004E0AA5E695E8A420CDA0626019F00F014
:107F4C00B7FD02982E520646052000077902002242
:107F5C0003F0DEFDA85B0028C0D0D8202858E98E9D
:107F6C008842BBDDE42028583C21695E7D22D2008A
:107F7C004A439042B2DDCE20295E4A22AB5E994242
:107F8C00ACDACC216B5EAA5E9342A7DA2A5E4E2055
:107F9C002B5E9A42A2DD695E285E81429EDDA85B63
:107FAC0002289BD00B4800F083FD0020A85301222F
:107FBC008EE7C04630000020B40F0020FFFF000009
:107FCC00EBC20008F4C40008B0C00008CAC2000824
:087FDC0010BF0008D2C000082C
:107FE400F0B581B076244A4D285B002804D0285B84
:107FF40001281BD101221BE046480088002846487E
:1080040002D041218900685241218E00A95B0029D8
:1080140002D0A95B81424CD1D8202858298F01274E
:10802400884200960FDD3D483E4637E0285B00223B
:10803400052000070121090203F06EFD285B354984
:10804400088001B0F0BDE42028583E21695E7D22FD
:10805400D2004A43904202DD022631481EE0CE207F
:10806400295E4022AB5E994202DD03262D4815E0CD
:10807400CC216B5EAA5E934202DD04262A480DE001
:108084002A5E44202B5E9A4202DA0526274805E040
:10809400695E285E81420CDA0626254800F00CFD54
:1080A40000982E520646052000073902002203F0EC
:1080B40033FDA85B0028C1D0D8202858698F884296
:1080C400BCDAE42028583E21695E7D22D2004A436E
:1080D4009042B3DACE20295E4222AB5E9942ADDAF9
:1080E400CC216B5EAA5E9342A8DA2A5E46202B5E00
:1080F4009A42A3DD695E285E81429FDDA85B022867
:108104009CD00C4800F0D8FC0020A85301228FE733
:10811400300000202A000020FFFF000024C50008D2
:108124000CC50008E0C000082DC3000833BF0008D8
:088134000CC3000802C10008A1
:10813C00F0B581B00A4D29688A09891A0E18B4095C
:10814C0008486043084901F0A7FC094F38802E60AD
:10815C000648214601F0A0FC788001B0F0BDC04675
:10816C00840F0020E8800000FFFF0000D08A2F75EC
:04817C00F8000020E7
:1081800010B586B01A480024FF217F22194B0360E6
:1081900001239B078460C260016144618461C46102
:1081A000036244620394029401940094FAF74EF837
:1081B000002801D003F093F901A98C7002200880F7
:1081C0000594049402940A480122FAF7F1F8002871
:1081D00001D003F084F9084800900548694601225F
:1081E00002F0D6FF002801D003F079F906B010BDE7
:0C81F000A00E002000280040010416181A
:1081FC0081B000680A49884201D001B07047012063
:10820C008102084A13680B43136013680B400093F8
:10821C000099C003116A0143116201B07047C04656
:08822C00002800403C10024054
:10823400F0B581B05821384E705A745ACF21490094
:10824400364D2F68775201F0A1FB354A354B03F0C8
:1082540066F901F0CFFAD8217658864202DD002073
:1082640028600DE0204601F091FB2F4A2F4B03F0CC
:1082740056F901F0BFFA86420ADA0020274908605D
:108284002B4908600120C043411C08B201B0F0BD75
:1082940027480168002906D00A460A32964208DDBA
:1082A40000211E4A0AE0066031460A460A32964216
:1082B400F6DC0A398E42194A06DA0021116001609F
:1082C400204908B201B0F0BD781C106019498842F9
:1082D400114D04D3E42028582321C90068522520D5
:1082E400C0002858144901F0DBFB144A136800212C
:1082F4009842CAD02323DB00EB5E114C2668B709F1
:10830400F61BF3189E098D277F00EE53106023603F
:10831400002001B0F0BDC046300000207C0F0020DA
:108324007B14AE47E17AF03F0AD7A3703D0AEF3FD2
:10833400740F0020312A000080510100780F0020C2
:08834400800F0020FEFF000085
:10834C0010B511494143C817000C081800146421DA
:10835C0041430E4808180A2101F076FB0C4A1146DD
:10836C00C831C88006200B5E08240C5F085EA3424F
:10837C0002DDD021505210BDD223D25E904201DAE0
:10838C00C888488110BDC046E40C0000A015FFFF52
:04839C00300000208D
:1083A000B0B5C1170A4D6A88002301F03BFB0622D5
:1083B000002301F037FB01F0F9FA044B002201F031
:1083C0001DF901F06DFAE860B0BDC046000024411F
:0483D000F800002091
:1083D40070B500210E480162416281620722C262C7
:1083E4000163416310230124A5041202094E0660AF
:1083F4004126B60046608160C2600246103232C235
:10840400C361FAF777F8002801D003F066F870BD6D
:08841400300D00200030014092
:10841C0070B58AB0002609960896079606960596BA
:10842C0000681A49884201D00AB070BD01242003AB
:10843C001749CA680243CA60CA6802400092009891
:10844C000868204308600868204000900996089648
:10845C00079602200690E02005900098052005075D
:10846C0005A92846F9F780F904960396029601941B
:10847C00E003009069462846F9F776F92021284652
:10848C00012203F045FB0AB070BDC046003001402C
:04849C003410024056
:1084A00082B009484168012211434160416811408E
:1084B00001910199110702680A43026000680840AF
:0C84C0000090009802B070473C10024091
:1084CC0010B5F7F7B9FE0B4C2068401C2060C008B3
:1084DC007D280DD3F7F7BCFE0749884208D307481F
:1084EC00C16D491CC16500212160816D491C8165EC
:1084FC0010BDC0466C0F0020214E0000F80000207B
:10850C0080B50248F8F7E4FD80BDC046F80D0020A8
:10851C0080B50248FBF7AAFC80BDC046A40A002027
:10852C0080B50248FAF7A6FC80BDC046540E002068
:10853C0030B501235902164801800246C832002189
:10854C00D16591654524A400CD43055355649564CC
:10855C004724A40005538F24640005532324E4000E
:10856C0005538D24640005530224048143810523A3
:10857C008381084B5C1C14625362074B5C1C148196
:10858C005381064C54619361C1225200815230BD1B
:10859C0030000020FFFFFF7FFF7F00000080FFFF07
:1085AC00B0B51E4D2C1F20688006400F411E0329BC
:1085BC0022D81B487944097949008F442301171AA2
:1085CC00296803220A40032A00D016482968490664
:1085DC00490F491C01F060FA29684904490E4843C7
:1085EC002968490F491C01F057FA0BE07D20000265
:1085FC0008E00120C00305E00C3D28688004410F11
:10860C000848C84008490860226892093C23134076
:10861C00064AD258D0400860B0BDC0460C1002408B
:10862C0000127A000024F400240000207CAF000823
:10863C00F0B587B000240694059404940394029436
:10864C0000681B49884201D007B0F0BD1948C168C9
:10865C000122049292031143C160C168114001913F
:10866C000199016802273943016000683840019084
:10867C000694059403974020029001980E4D02AE8B
:10868C0028463146F9F770F806940594049403973C
:10869C008020029028463146F9F766F81B2000210D
:1086AC000022F8F7ABFB1B20F8F7C4FB07B0F0BDBA
:0C86BC000038014034100240000400505F
:1086C8000548016E054A4A432921C900425040180D
:1086D800D11741607047C04630000020F0F1FFFF1D
:1086E800F0B589B0664A0ACA0846083A184307D15D
:1086F80000234D20800063490858634941430AC25A
:108708000191624A12CA0846083A204307D1002458
:108718002720C0005B4908585B49414312C20391B6
:108728000494E420574C2158002902930ED4722156
:10873800615A20584843642101F088F95F21890073
:1087480060507020205E6158081A01E0F02020581F
:108758005F21890060506258D317D8202058C1176C
:1087680001F05CF97D22D20000230092079301F00A
:10877800B9F917221501059566190896276E7268CA
:108788006359C31863514A4172602922D200A31861
:108798005C683C4DAE583018A8504C415C60E120F4
:1087A8000401380C00260694A4B26043BFB27C438F
:1087B800050C000421187541324E00200024611870
:1087C8006841089C6468059FF5594D1B0546A541FD
:1087D8003C4602DA3151089948605868B158491E38
:1087E8000799884101DBB1505960B0585968002396
:1087F800069D2A4601F076F95B21890070503059B0
:10880800089949682A46002301F06CF92F21C9000C
:1088180070502120C00031583058002912D4C11797
:10882800039A1418049D4D41174A002320462946EF
:1088380001F070F92721C9007050144804604560A0
:1088480009B0F0BD4042C117019A1418029D4D416C
:108858000D4A00232046294601F05CF93146C8310B
:10886800C866496E00984843F16D01F017F94F2129
:108878008900705202480460456009B0F0BDC046E6
:10888800A80500203000002080EE3600B00500204A
:10889800F0B581B05B208000184C21582058002981
:1088A80000D540422146C8318864496C14480029E3
:1088B8001ED44321890061587D22E36D994216D266
:1088C800E36D002B14D0D00000230A0C002680B2E0
:1088D80042438FB27843150C1104401875410021AA
:1088E800002210186941E26D01F014F900E0D0008F
:1088F80045218900605201B0F0BDC046300000201B
:04890800FFFF00006D
:10890C00F0B581B01149086E00281CD0E12212018B
:10891C000023040C002692B2544380B24243270C2D
:10892C002404121977410024002085187C4117205B
:10893C000201885889184968054A01F06DF82A46E1
:10894C00234601F0CDF801B0F0BDC0463000002048
:04895C00A0860100F0
:10896000F0B581B05B20800016490A58002A01D476
:10897000002001E008584042112212018B58002BC0
:1089800002DD8D58EE1701E00D6E0026C1170E4F67
:108990007A1C0024234601F045F82A46334601F0AC
:1089A000A5F802460948BB1A23468B4103DA002981
:1089B00004D501B0F0BD841A0029FAD4204601B0D4
:1089C000F0BDC046300000209F860100A086010057
:1089D000F0B581B0112003011E4AD058002808DDEF
:1089E0004320800010582D21C90051580818C11784
:1089F00005E0D06D2D21C9005158081800211446FA
:108A0000C83426690325ED01575BA46C012C02DBF9
:108A1000D458E51701E0146E0025F219D30FD318CE
:108A20005A10DB1700F0FEFF7D22D200002301F078
:108A30005DF8094E3246002300F0F4FF22462B4633
:108A400001F054F8C1178843B04200DB304601B052
:0C8A5000F0BDC04630000020A0860100F0
:108A5C0070B51248026EE1210B010021140C0026A6
:108A6C009BB25C4392B25343250C24041B197541F1
:108A7C0000240022D2186C4117231B01C250C218CB
:108A8C0054602922D2008150821851605B229200DE
:108A9C00815009225201815070BDC0463000002027
:108AAC0080B50249096803F08DF880BD18000020DC
:108ABC00B0B5044608480568204602F01FF9024686
:108ACC002846214602F037FE401C03D00A20FFF74F
:0C8ADC00E7FFB0BDC043B0BD1800002093
:108AE800C20F490089184000034A40428A4101D315
:0C8AF80000207047012070470000E0FFE4
:108B04000122D2079143034A4A401043414248415B
:088B14007047C0460000F07F2D
:108B1C00074A0A40531E9A41C00F490008180549DC
:108B2C00884201D300207047012010407047C04696
:088B3C000000F07F0000E0FFE3
:108B440030B50E4B5D1C0C0D2C4011D0AC420FD037
:108B5400A2189A4206DD0120C007014009480918FD
:108B6400002030BD002A04DD054B194012051143D5
:108B740030BD0120C0070140002030BDFE070000C9
:088B8400FFFF0F800000F07FED
:108B8C0010B54B005B0D084CA34201D0002B02D159
:108B9C000023136010BD054C1B191360044A1140CF
:108BAC00044A891810BDC046FF07000002FCFFFFF5
:088BBC00FFFF0F800000E03F05
:108BC400F0B587B00025EC43584E0494671C344636
:108BD40000956C415D0003956D0D554D059577D05D
:108BE4000297C50F06914F0001977F19450004991C
:108BF4004D1BBE416CD3D50F03994D1956000299F4
:108C04008E1BAC4164D30125EC0706990C400594F6
:108C1400484C0E4626402340141A1C46B44175D2D3
:108C24002C05019F7F0D0494039505D02546641EF1
:108C34000E4626402E430BE0A64209D2E9043446F0
:108C4400C50F6600761940007F1E8C423446F7D368
:108C5400190D394C214006D0049D6C1E23402B4332
:108C64008F4221DC2AE004998B4210D20399C90473
:108C7400069100211C46D30F6500EB185200491ED3
:108C8400069DAC421C46F6D38F420DDC16E0002153
:108C9400002F09DC12E005463446E80F640026186C
:108CA40068007F1E8F4208DD851A34469C41F2D449
:108CB40050405E400643F0D10AE00F460546A81A2C
:108CC40031469941049C05D455405E402E4303D15E
:108CD400009818E02846314621420AD1039DEA044F
:108CE400C30F4C00E31840007F1E11421946F7D011
:108CF40001E00B46039D002F11DD791E059A9A1899
:108D0400090551180591059907B0F0BD42405E4030
:108D1400164300D00591002EF5D10020F3E7EA1B9D
:108D240000F05EFE0B460021E8E7C046FFFFDFFFD0
:0C8D34000000F87FFFFFFF7FFF0700003A
:108D4000F0B583B00C462A494B1C220D1A40531E25
:108D50008B4242D228498A4206D20020002C01468A
:108D600039DA284903B0F0BD33318A4202D92146AD
:108D700003B0F0BD1F495518029021462A4600F065
:108D800021FE1E4A11400143484248410027002C61
:108D900001DA394600E001210143019118493846C2
:108DA0002A4600F02FFE2A4605460E462640029827
:108DB0000540F843401C1149794100F013FE0A4672
:108DC0003146019C2B187241002C00D11146002C19
:108DD00000D11D46284603B0F0BD002A02D1012172
:108DE000C9070C402146002AF5D1002003B0F0BD90
:108DF000FE07000001FCFFFFFF030000FFFF0F0064
:088E00000000F0FF0000F0BFCC
:108E0800F0B587B00A0D521E494B9A4212D206AAF3
:108E1800FFF7B8FE4B4A821A494A0B469341069C13
:108E28001CDA0022494B00F0F9FA641E0594044646
:108E38000D461EE0C30F4A00D318440064423D4C5F
:108E48009C416FD3520D6FD000290A4600DA3B4A85
:108E5800002900DA0020114607B0F0BD00223A4B85
:108E680005460E4600F0DAFA0594044628460D46F3
:108E780031460026F2430496FFF760FE344B002289
:108E880000F0CCFA02460B462046294600F0B2FB19
:108E980003900F4602460B4602F03FFB04460D4680
:108EA8002C4E0221304622462B4602F0BBFE2A4AAF
:108EB8002A4B00F0B3FA0290019110360321304694
:108EC80022462B4602F0D6FE02460B46029801992E
:108ED80000F090FB22462B4602F01FFB039C224623
:108EE8003B4602F01AFB22463B4600F097FA06463C
:108EF8000F46059800F00CFD04460D46184A194B1C
:108F080002F00BFB32463B4600F088FA06460F4655
:108F1800154B20462946049A02F0FFFA32463B4692
:108F280000F07CFA07B0F0BD0349002007B0F0BD9F
:108F3800FE0700000000E0FF0000F0FF0000F87FDF
:108F48009EA0E63FCE3B7F660000F0BF0000E0BF7A
:108F58000000E03FC00000089AB5B312FF0750C0F8
:0C8F6800A80C615C10D02BBF0030E63F6D
:108F7400F0B585B05B4A531C0C0D1C40631E934234
:108F840000D393E05B4A121A594A8A4100DAA7E0F7
:108F940000235A4A121A584A8A411A4600D281E0DA
:108FA4000122D2070B469343574A821A554A9341EA
:108FB40076D3564A564B02900D4602F0B0FA01227F
:108FC400D2072A40534BD31800242246049400F0BD
:108FD40027FA00F00FFC039000F09CFC06460F46B5
:108FE4004D4B002202F09BFA029A2B4600F018FA2D
:108FF40004460D46494A4A4B3046394602F08FFA38
:1090040022462B4600F00CFA06460D4602460B4655
:1090140002F085FA0746434A434B0C46029102F09C
:109024007EFA424A424B00F0FBF93A46234602F0EC
:1090340076FA404B049C224600F0F2F932462B4665
:1090440002F06DFA05460E46204632492A4633465A
:1090540000F0CAFA01900091374A384B3846029C16
:10906400214602F05CFA364A364B00F0D9F93A460A
:10907400234602F054FA019A009B00F0D1F902460B
:109084000B462846314600F0B7FA049A214B00F00B
:10909400C7F9039A521CFFF753FD03460A4601E041
:1090A400174A00231846114605B0F0BDC20F4B0005
:1090B4009A1843005B420C4B9341EED30122D20732
:1090C4000B469343094A5A40024300D071E70029F2
:1090D4000A4600DA0022002900DA00200346E1E70C
:1090E400024ADEE7FE0700000000E0FF0000F07F18
:1090F400422E8640EF39FAFE2B2386C0D2BC7ADD9D
:109104000000F03FA19CC73B2342920C3CF92F9EE8
:109114002C15F73F0000E03F0030E6BFA80C615C6F
:1091240010D02B3F1CDC586FA452F13EE0F6B36F15
:10913400E4707C3F0000D03F0938DE6F993F403F28
:08914400B35142718E71AC3F82
:10914C00F0B587B01E460B4604460020C743924D2F
:10915C00791C2946414159400294214300D1A9E090
:10916C007400610D8D4900D112E1039704950692AC
:10917C008C4F7A1E05935D006B0D5B1E934273D270
:10918C00320D3A40884BD218521E9A426CD3069834
:10919C00314600F02BFB074600F0B8FB012204928D
:1091AC00D407A742059D32D0069A50407140014326
:1091BC002DD1002F019745D0F81747403E1A774F15
:1091CC000024039402980BE0424222400698394650
:1091DC0002F0A1F904460F4676082846059D33D0C7
:1091EC00012E039A00D002460694012E6B4B00D040
:1091FC002B460446294602F08EF92A46054605916F
:10920C00304604990840654BDED01346DCE70496E3
:10921C000022029E304629462F46134600F0C6FA1D
:10922C00002803D06549002007B0F0BDA7433046A5
:10923C003946FFF7E3FD069A049B02F06CF9FFF741
:10924C0093FEA5E0554F00240020544922463B468E
:10925C0000F0CEF9019A002A00D43946002A00D534
:10926C0096E0204607B0F0BD3746029EF20FAA18D2
:10927C0073005B1E4E4B534120D20125069EF20F0C
:10928C00A21873005B1B494B9A411BD2444A059BA5
:10929C0013421BD0474C1A466240029E324332D0D6
:1092AC001A463F4B5A40324348D1002F5BDA0146F5
:1092BC0007B0F0BD2046194607B0F0BD3046059901
:1092CC0007B0F0BD3046394607B0F0BD30463E46DB
:1092DC000446394600F08AFA074600F017FB32467E
:1092EC004A4023464340134300D057E70021002E49
:1092FC00084600DA2A49FA074AD0EA07059B1340C8
:10930C00591807B0F0BD0490002F00DB24480590DD
:10931C00069C20463E46394600F068FA074600F0A7
:10932C00F5FA714060400843059802D1E8070599A9
:10933C000818F90700D005900498C0E76740069A12
:10934C003A4313D11C4A059B5A40334632431FD033
:10935C00E807059A824300211846039B181A0498C3
:10936C009041084614D30E4907B0F0BDE8070599A3
:10937C0081430020039B9A1B049A8A41014607D221
:10938C000D48059941403046084303D004494AE74B
:10939C0007B0F0BD014946E7FFFFEF3F0000F03F8B
:1093AC000000F07FFF07000002F8FFFF0000E0FF65
:1093BC00FFFF1F000000F0FF0000F0BF0000F87F6F
:1093CC0070B5040011D0E017214641400D1A104928
:1093DC000020104E02E008366D0807D0EA07FAD0DC
:1093EC000CCE083E02F097F8F5E70949084E024604
:1093FC0000200B46314616461D4600F0F9F8002CAD
:10940C0001D502D570BD3046FCD4294670BDC0468E
:08941C000000F03FE800000829
:10942400F0B40125ED070F005F405AD48B4200D100
:10943400824205D950404240504059404B40594027
:109444004E18760DDF187F0D3BD0741C640529D0AF
:10945400F41B352C26D80E0DDB022B43DB0AC90284
:109464002943C9121700202C1ED2E741E24057407D
:10947400E3415A40A340E3405A4000248018594134
:109484000AD3B21C520521D0C207012F6241170032
:109494004008CB0718434908013636054208AF4156
:1094A40060417141F0BC7047203C06D01F00E74189
:1094B400E3405F400024012A6741C0186141EBD3B7
:1094C400DFE7002EEED129400020EBE7013631051D
:1094D4000020E7E7E742E5D10020C143090DC904B4
:1094E400E0E76B400E00871A9E4104D26E40C01B19
:1094F400B141D21973414E18DF18AC0AE642E9D2E1
:10950400760D7F0D31D0F41B362CCBD8B4460E0D1E
:10951400DB022B43DB0AC9022943C90A012C32D8D6
:1095240004D1D4075208DF073A435B08EF0A6442C8
:10953400904199411ED0002239424DD12419404115
:1095440049410124394204D10134001849413942C6
:10955400FAD06246A24204D9361B013E3605891967
:10956400A0E7F10AC90700209CE736429AD10020FF
:10957400002197E70200224394D0B842DED20100D2
:1095840020002024E3D1202C13DD203CE2411700ED
:10959400A240E2405740E3415A40A340E3405A40CE
:1095A400012FBF410137174300227C42984191416A
:1095B4000CE01700E741E2405740E3415A40A34022
:1095C400E3405A407C429041994100220F0303D268
:1095D400013E241940414941013E36054708AC414A
:0895E40050417141F0BC7047D9
:1095EC00F0B40125ED076B40004C20472B9400088C
:1095FC00F0B40125ED070C005C402C40A446AE0AEB
:10960C004C18DF18F4423DD2F74245D2640D4CD0D1
:10961C007F0D3CD0E41BC9022943CF0ADB022B434C
:10962C00DB0A0600B61A9F4104D2013CB6197F41F1
:10963C00B6185F416812800D241838DD001884427A
:10964C0025D8E80C0021B6197F41B61A9F4103D3E7
:10965C0040414941F7D304E0B6185F410018494135
:10966C00F1D32405B6197F41B61A9F4105D3374370
:10967C00C20717430022012F50416141624611433A
:10968C00F0BC70470CD100280AD1F74208D2002058
:10969C00C143490D0905F1E7002A01D1F74206D073
:1096AC000020C143090DC904EAE77F0DF8D0002062
:0496BC006146E5E737
:1096C00030B401256D054C00E54215D85C00E5423B
:1096D00012D80C001C436400044314430FD005D27D
:1096E00082428B418041013030BC704790429941A9
:1096F0008041013030BC7047002030BC70470120F1
:0497000030BC7047C2
:1097040070B4012676054C005D00E6420CD8EE42AA
:109714000AD825430543154303D0994204D1904206
:1097240002D1012070BC7047002070BC7047C04655
:1097340030B401256D054C00E54215D85C00E542C6
:1097440012D80C001C436400044314430FD005D208
:10975400904299418041013030BC704782428B4134
:109764008041013030BC7047002030BC704701207C
:0497740030BC70474E
:1097780030B401256D054C00E54215D85C00E54282
:1097880012D80C001C436400044314430CD005D2C7
:1097980082428B418041404230BC7047904299419F
:1097A8008041404230BC7047002030BC7047C04602
:1097B80030B401256D054C00E54215D85C00E54242
:1097C80012D80C001C436400044314430CD005D287
:1097D800904299418041404230BC704782428B415F
:1097E8008041404230BC7047002030BC7047C046C2
:1097F800F4464A1805D200F051F801D5C0174008C0
:10980800604701235B05D34206D200F047F801D533
:109818000120C0074042604701D10042F5D0D0176F
:04982800400870473D
:10982C004A00520D01239B02D21A01321DD452421E
:10983C003F321DDD8C46C902430D1943C002012382
:10984C00DB071943202A02D308000021203AD1411A
:10985C00D04048409140D140484063461B4203D51C
:10986C00002340428B4119007047002000217047B3
:10987C00002801D0012211434B0001225205D34292
:10988C0000D959080020C90FC90701D4C0434108A9
:04989C007047C0460B
:1098A0004A0010D2520D03231B02FF33D21A0AD4EE
:1098B00052421F3209D4400DC90208430123DB077D
:1098C0001843D040704700207047D0177047C046FB
:1098D0004B001BD25A0D01239B02D21A013215D420
:1098E00052423F3215DBC902430D1943C002012326
:1098F000DB071943202A02D308000021203AD14176
:10990000D04048409140D14048407047002000215D
:089910007047D01701007047F9
:10991800054B004206D5404200B5984708BC0122D5
:0C992800D2071143184700009199000875
:109934000B00034329D0CA0FD200043212023D3275
:10994400094203D5002349424042994102D1010012
:109954000020203A0B0C04D1103A0904030C1943DB
:109964000004094203D4013A00184941FBD5844656
:10997400C00A4B051843C90A120563465B055B41DF
:0C99840002D3012B0023584151417047D1
:1099900042221201033A010007D002D4013A001812
:0C99A000FCD51205C30A40059918704759
:1099AC000B00034305D0042212023D320942014B45
:0899BC0018477047519900089B
:1099C400202A07D203009040914052422032D340D3
:1099D40019437047203A0100914000207047C04667
:1099E400202A07D2D0400B00D1405242203293406B
:1099F40018437047203A0800D04000217047C04601
:109A0400202A07D2D0400B00114152422032934009
:109A140018437047203A08001041C9177047C046E0
:109A240030B5514343435C18010C130C0D005D43E6
:109A3400641992B2514380B242430D0C0904521886
:109A440065415843010C00048018694130BDC0468B
:109A5400CA1751408B1A17D0C1174A409446484040
:109A6400411A48081A0000E052008242FCD9002042
:109A740000E05208914200D3891A40419A42F8D139
:109A840062465040801A704710B500F095F810BD3A
:109A940007B5FFF7DDFF0EBC4243891A00BDC0467F
:109AA4000A0015D00300400800E052008242FCD9AD
:109AB400002000E052089B1A06D340418A42F9D1A3
:109AC400704752089B18F8D200188A42F9D170479F
:089AD40010B500F071F810BD9F
:109ADC0038B504004D42FFF7DFFF4543611938BD2F
:109AEC0070B5CC1760406140001BA141DD176A4086
:109AFC006B40521BAB4100F00BF862406340121BF1
:109B0C00A3416C4060406140001BA14170BDC04648
:109B1C00002B09D1002907D110B51100FFF7D8FF90
:109B2C000A000021002310BD70B400240125ED07AC
:109B3C00002B07D1002905D0834203D21300002249
:109B4C002C0000250026A419994200D1904212D96C
:109B5C0092185B4103D2EE076D086408F3E7DE0749
:109B6C005B08520892190126F6079B1903E0DE07E1
:109B7C005B0852089219801A994103D364416D41D4
:109B8C00F5D30FE024196D410AD2DE075B085208A9
:109B9C00921980185941F5D364416D41E7D301E026
:109BAC008018594102000B002000290070BC70473E
:089BBC00002000217047C046A3
:109BC400F0B503AF93B06E46F51D2135F41D39345D
:109BD40074613362F261F160306102F0A5F8B06043
:109BE400C21D07218A436946B1616946881A7060BB
:109BF4008546F41D1D3400212422204601F050F92D
:109C04000B487169F2680A6048600A482860306944
:109C14002862B06868617068E8602046F169326A59
:109C240000F01EF8B1698D46FE1F053EB546F0BD35
:089C34001DBD0008FFFFFF7FCA
:109C3C0083B010B581B0044603A80EC00548006877
:109C4C0003AA0092214601F069FD01B010BC02BCD0
:089C5C0003B0084718000020C6
:109C6400F0B59FB011921691064600203060012194
:109C74000A020E924A020B928A020192CA020092CE
:109C840003220D92920205920A0317924A03069246
:109C94008A0304920391C9030990C0430290149665
:109CA4000D460A9102E0304601F0E2FC1698017874
:109CB400252906D0002901D100F07BFF401C169015
:109CC400F1E7C01C099E0B9C0746801E00780246E3
:109CD400203A3E2A00D940E08021C0467A441279D5
:109CE40052009744233A3A203A3A3A293A3A2D2BE9
:109CF4003A1F3A3A253A3A3A3A3A3A3A3A3A3A3AF0
:109D04003A3A3A3A3A3A3A3A3A3A3A3A3A3A3A3AAF
:109D14003A3A3A3A3A3A3A3A3A3A3A3A3A3A3A3A9F
:109D24003A3A270010210E43781CCDE74021FAE788
:109D34002146F8E71799F6E72946F4E72021F2E7E8
:109D4400119901C91191C10F09010E43C11748406E
:109D5400441A3A46781E007810E07A1E01463039DB
:109D6400002409290AD80A2161434418303C511CB3
:109D740010780246303A0A2A0A46F4D300232E28E1
:109D84000AD110782A28374609D15078921C1199A3
:109D940008C91191149E13E03746149E14E0521C16
:109DA400014630390929149E0CD80A215943431815
:109DB400303B511C10780246303A0A2A0A46F4D342
:109DC400002B01D40E990F43169201464C392E29CB
:109DD40039D849007944898849008F442E003400D9
:109DE40034003400340034003400340034003400CF
:109DF40034003400340034003400340034003400BF
:109E040034003400340034003400340034003400AE
:109E1400340034003F0134002E0034003901340092
:109E24003400340034003400340034003000340092
:109E34003400340034003400300002200743169903
:109E44000878491C1691782800D92FE7E1178C432C
:109E5400810001A251588F46D5AB000845A00008E7
:109E640045A0000845A0000845A0000845A000083A
:109E740045A0000845A0000845A0000845A000082A
:109E840045A0000845A0000845A0000845A000081A
:109E940045A0000845A0000845A0000845A000080A
:109EA40045A0000845A0000845A0000845A00008FA
:109EB40045A0000845A0000845A0000845A00008EA
:109EC40045A0000845A0000845A0000845A00008DA
:109ED40045A0000845A0000845A0000845A00008CA
:109EE40045A0000845A0000845A0000841A00008BE
:109EF40045A0000845A0000845A0000845A00008AA
:109F040045A0000845A0000845A0000845A0000899
:109F140045A0000845A0000845A0000845A0000889
:109F240045A0000845A0000845A0000845A0000879
:109F340045A0000845A0000845A0000845A0000869
:109F440045A0000845A0000845A0000845A0000859
:109F540045A0000845A0000845A0000845A0000849
:109F640045A0000845A0000845A00008D5A00008A9
:109F740021A10008CDA0000845A0000845A00008C4
:109F840045A0000845A0000845A0000845A0000819
:109F940045A0000845A0000845A0000845A0000809
:109FA40045A0000845A0000845A0000845A00008F9
:109FB40045A0000845A00008DDA0000845A0000851
:109FC40045A0000845A0000845A0000845A00008D9
:109FD40045A0000845A0000845A0000845A00008C9
:109FE40045A00008A7A0000847A00008D9A00008C1
:109FF40025A10008D1A0000845A0000847A000083A
:10A0040045A0000845A0000845A0000845A0000898
:10A0140003A100088BA00008C9A1000845A00008FE
:10A0240045A00008C1A1000845A00008E9A1000856
:10A0340045A0000845A00008E1A00008252132E65B
:10A0440034E61E4604990F4300210891394626E060
:10A05400169908786C280AD1022004E01699087829
:10A06400682808D1082007434878891CEAE6491C77
:10A074001691039902E0491C169104210F43782894
:10A0840000D8E3E612E61E460E990F42394601D087
:10A09400D14A11403A06D217302313400893119D38
:10A0A400AAE03D463746119E30781590641E384626
:10A0B4002946224601F01AFE38462F46159901F02A
:10A0C400D7FA361D119602E106980743059828E051
:10A0D40006980743019824E006990F43BF4A78285D
:10A0E40000D12032119D1E460E990F42394601D0EF
:10A0F400B94B19403B06DB17134008937CE0119AD7
:10A1040010683907316800D55FE2BA07016001D5EC
:10A11400002141601198001D1190C7E5069807437E
:10A12400009807430E98074200D106230C94394641
:10A13400059A1140891A4A424A41002B00D01A4616
:10A144001592119CE41D07208443266865683046F7
:10A154002946FEF7D5FC08341194002812D00022B9
:10A16400304629461346FFF725FB3A4606990A402E
:10A1740000280C9C17D0002A9948159B00D180E038
:10A1840098487EE030462946FEF7ACFC00280C9C3B
:10A1940000D1A7E006980742934800D09348944919
:10A1A4000F40159B6FE0002A9249159B00D09249FD
:10A1B400002A62D09148BA0662D462E0119901C9BA
:10A1C400119160E00C9438060E990F430F97C01755
:10A1D400232101400891119808C8119000270820F4
:10A1E400079011E10E991E460F4201D07A490F40A3
:10A1F4003946119D0022089202220A40049B19420A
:10A204000C9406D1002A0DD12B1D00272A461D4689
:10A214000EE0002A18D104CDD7174B071BD513B273
:10A224001204A3E0EA1D07239A435768154608352C
:10A2340013684A071ED408220A4000D0DBB2002A61
:10A2440000D19EE000279CE0ED1D0722954384CDBC
:10A2540000354B07E3D40B0700D585E01346002FE8
:10A2640000D486E000225C42BA412D2308932346A1
:10A27400174686E09BB2002783E06148BA0600D502
:10A2840008465B490F4000285E4E00D006460E98F3
:10A29400074203D1304600F035FD03E0304619464D
:10A2A40000F084FD05464C480740641B1498394669
:10A2B400224601F01BFD002D09D00F97149F317821
:10A2C400384601F0D5F9761C6D1EF8D10F9FF806BB
:10A2D4000A9D149E00D4E9E420213046224601F070
:10A2E400F7FCE3E430462946FEF716FC002800D1CB
:10A2F4000646002800D100253046294601F092FC8C
:10A3040004460120002C089001D0C00745401EAA35
:10A31400304610952946FEF737FC1E980D994843A0
:10A324000A21FFF795FB05461E90002C129601D0DA
:10A334006020074300223046109C214613921346A6
:10A34400FFF7DEF9002800D023E1681CFFF73CF892
:10A3540032462346FFF72EFA002800D10CE11E985E
:10A36400411C1E91801CF1E753B21206D71700D589
:10A3740078E78A0603D44A0603D5202200E02B227C
:10A3840008920E9A114201D0134A11400A461195BF
:10A394000E990F920A42039900D03146079158381A
:10A3A400002420280A9A00D997E0C046784400790E
:10A3B400400087442992929292929292929292921F
:10A3C40047929292924792929292927C299292927E
:10A3D400924792922900C046FFFDFFFF58300000CB
:10A3E40053C300084EC3000868C5000864C50008CC
:10A3F400FFFEFFFF5DC3000858C3000859C30008EF
:10A404005EC3000856BF0008184638434DD006986E
:10A414000F990142F64800D0F64819093A078918FD
:10A4240000240A460F211940415C18AB1955110943
:10A434003F093B07C91813463B43641C002B1346D2
:10A44400EFD14AE01846384347D00F981040109097
:10A454001EE015940A2200251846394613971293D4
:10A464002B46FFF759FB04460F460A222B46FFF7FB
:10A47400D7FA2346129C201A3021014318A8159AB2
:10A484008154521C0920001B13988541144624D280
:10A4940010980028DDD020460D9908400328D8D113
:10A4A40018A82C210155641CD3E7002415E0184694
:10A4B400384312D0D80879074018014607201840BD
:10A4C400303018AA1055C808FF087A0780180A46C1
:10A4D4003A43641C002A0B46EFD1089DFF2D01D896
:10A4E400029801E0C448FF300B9F0C9B07990E1B98
:10A4F400F1178E431594A1195A1A002D00D0121881
:10A504000F99394203D1149801F0F0FB0022139201
:10A51400290A04D0149C204601F0AAF802E0002D78
:10A52400149C03D02046294601F0A2F820460F9936
:10A53400139A01F0DBFB30212046324601F0C8FBC0
:10A54400159F012F0ADB7D1C18A84019801E017875
:10A55400204601F08DF86D1E012DF5D80F98C00628
:10A5640026460A9D01D4FFF7A1FB20213046139A09
:10A5740001F0AEFBFFF79AFB1E98FEF725FF32466B
:10A584002346FFF7F7F8002803D01E98401E1E90BC
:10A59400F3E73D4605980540089883021E989D42BE
:10A5A400159E17D005998D4205D1864212DD0421EE
:10A5B400C94388420EDD01990F42109D0F9300D1CB
:10A5C40077E10E2838DD139E73E10170121D11929C
:10A5D400FFF76CFB0E9934318842109C079506D125
:10A5E40012982146854A864BFFF706F806E040425A
:10A5F400FEF7EAFE129A234600F091FF04460E4647
:10A6040000221346FFF77CF8002813D12046314678
:10A61400FEF776FA002837D000222046314613464A
:10A62400FFF7C8F83A4606990A40002800D104E129
:10A634000C9CA0E50F9759E0C143711810290E46F0
:10A6440000DB10263A0600D533E1002900D130E1C1
:10A654003046FEF7B9FE129A2B4600F060FF002444
:10A664002246684BFEF7DCFEFEF768FB2246664B8B
:10A67400FEF7A6FA22462346FFF742F8002800D147
:10A6840014E1761EE4D112E10F97002220463146F0
:10A694005D4BFFF74DF800281E9F0FD00022204687
:10A6A4003146594BFEF7A8FF04460E460022564B8E
:10A6B400FFF73EF87F1C0028F0D11E9700222046A9
:10A6C4003146524BFFF776F800280FD0002220467F
:10A6D40031464D4B00F023FF04460E4600224B4BFF
:10A6E400FFF768F87F1E0028F0D11E970598079998
:10A6F400814202D01598014601E01598411E0028B8
:10A70400139100D100210F464842FEF75DFE029AE4
:10A71400FEF716FA22463346FEF782FE06460D463B
:10A7240000221092384C2346FFF702F800280AD082
:10A734001E98401C1E900022304629462346FEF7F0
:10A744005BFF06460D4612961595002F2CD00099F6
:10A75400084680300F9A1040884227D1102F00DB22
:10A7640010273846FEF730FE32462B4600F0D7FE5F
:10A77400FFF7ACF8024608431098139016D00C4625
:10A7840010461646224A234BFFF74AF94A08C307E4
:10A794009A184008C90708181F49081A1F48904109
:10A7A40000D3F0E1139701E01098139080210F98E3
:10A7B40006460140139A11430C98801A002901D1CE
:10A7C400471F00E0871F17981E9C064201D1089D71
:10A7D4004AE0032120461091FFF75AF9881C01250D
:10A7E40078440079400087441B2F3B1B2F00C04650
:10A7F40054C5000844C50008FFFEFFFFA0C8EB8550
:10A80400F3CCE17F0000E03F000024400000F03F73
:10A81400CDCCCCCCCCCCCCCC99999999999999198B
:10A82400641E1E94002212981599ED4B00F077FED9
:10A83400129015917F1E022512E0002AE7490C9C14
:10A84400159B00D0B3E4B3E4A41E1E940022129816
:10A854001599E44B00F063FE12901591BF1E109DF4
:10A864001399C817814313917006800F00D07F1E7F
:10A874001097204601F028FA632801DD781E109015
:10A884000898C0023746874312981599FFF71EF8B7
:10A8940004460E46FFF788F802460B4612981599AF
:10A8A400FEF7A2FE15901291109A75E034461E9898
:10A8B400264610387142884200DC0846FEF784FDC3
:10A8C400029AFEF73DF9129A2B46FEF7A9FD0546BA
:10A8D4000C461E98401CFEF777FD15952A46234624
:10A8E400FEF7ECFE00281E9800D0401C00281396AA
:10A8F40014D4112817D3014610391E911021081AB7
:10A90400FEF762FD2A46234600F009FEFEF7DEFF4D
:10A9140004460E4600201290159017E0129400246D
:10A924001E94264612E000201E9028462146FEF77B
:10A93400CDFF129404460E46FFF736F802460B4646
:10A9440028461299FEF750FE1590129138460F9939
:10A954008843A64900250A4608326D1C0B684968DD
:10A96400E31A33468B411146F6D280213940139ABB
:10A9740011434B1E0A469A41002901D00021C943C4
:10A984007B069B0F00D0D1431E9A891A0C9A139B05
:10A99400D21A51184A1B0746D017114681430B9807
:10A9A40010300F9707420AD1012A08DB0F462021F5
:10A9B400149800F05DFE7F1EF9D10F9A01E03A462B
:10A9C4000F4640201040910603D4002809D02021CE
:10A9D40004E0002801D02D2100E02B21149800F080
:10A9E40047FE0F98C0060FD4002F0DD030211498C5
:10A9F40000F03EFE7F1EF9D106E03020C1B214986B
:10AA040000F036FE002D12D06D1EE800764A1118B3
:10AA140049681258A01A30468841EED33020A41A4F
:10AA24008E41401CA31A33468B41F8D2E6E71097B7
:10AA34000F9D2C4600980440149E0BD01E980128AC
:10AA440008DB401E1E903021304600F011FE1E9897
:10AA54000028F6DC80202840139F384346D02E215E
:10AA6400304600F005FE102F3D463E4600DB102523
:10AA7400E8178543002C01D1284601E01E98281AC6
:10AA8400129CFEF7A1FC012E23DB159A234600F04D
:10AA940046FDFEF71BFF04460E462F4606E0302017
:10AAA400C1B2149800F0E4FD002F12D07F1EF8000C
:10AAB4004D4A111849681258A01A30468841EED3FD
:10AAC4003020A41A8E41401CA31A33468B41F8D27D
:10AAD400E6E71399481B149E28460F9D06D0441A96
:10AAE4003021304600F0C4FD641CF9D301980542BE
:10AAF40029460A9D109F30D00698014201D0452175
:10AB040000E06521304600F0B3FD1E98002830D4E3
:10AB14002B21304600F0ACFD1E9864280DDB642127
:10AB2400FEF7BEFF01463031304600F0A1FD1E980D
:10AB34006421FEF7ADFF08461E910A21FEF788FF47
:10AB440001463031304600F093FD1E980A21FEF78D
:10AB54009FFF3031304600F08BFD002F01D1FFF70D
:10AB6400A5F82021304600F083FD7F1EF9D1FFF7C0
:10AB74009DF82D21304600F07BFD1E9840421E902A
:10AB84006428CCDAD9E7139730460A2200232146F9
:10AB9400FEF7C2FF0C4607460A220023FEF7BCFF5D
:10ABA4001398401E139000D100E61A433846ECD0A7
:10ABB400FCE5F068002805D006CE083E914201D29B
:10ABC400099A4254304600F0A0FD30681FB0F0BD31
:10ABD400304600F09AFD02981FB0F0BD5DC3000836
:10ABE40000002440000059403001000838010008EA
:10ABF40009490968091A4A1E9141084A1268121A39
:10AC0400531E9A410A4006490968081A411E8841A0
:10AC1400104040427047C046180000201C0000202D
:04AC240020000020EC
:10AC280070B5182343431848C318DD6A184618300E
:10AC3800022D10D0012D08D00024002D21D15E6AEC
:10AC48009D6AB54214D9F34315E05D6A9C6AAC422B
:10AC580005D9EB4306E000F092FD004670BDED43D8
:10AC680064191B6AE418944200D31446224606E08D
:10AC7800F643AD191B6AEB18934202D3144600F051
:0CAC880061FD204670BDC046FC090020A4
:10AC940070B50B4616490C78002C1DD103240C61A9
:10ACA4004C61144D8D61144CCC610124A4020C62DE
:10ACB40000248C624C62CC620D66104D4D661025EA
:10ACC4008D660C67CC664C670D4D0F266640AE5DF5
:10ACD4000E55641C102CF8D1EFF31084012181F37C
:10ACE40010881946FFF79EFF84F3108870BDC04694
:10ACF400FC09002073C30008BA0F00203A14002096
:04AD040062C300081E
:10AD0800F0B582B0017800292FD0032201460092C5
:10AD180091430D6800220192D4438607F60EB44091
:10AD2800E4432C431E4D6719A7431E4B1F4222D1F3
:10AD380008310F1F3C6862191E46A643164217D1F8
:10AD48000C6862191E46A643164214D14C68621953
:10AD58001E46A64316420DD18C6862191E46A643AC
:10AD680010311642E5D0083905E0002002B0F0BDE8
:10AD7800394600E0091D2206019A0DD02204120E60
:10AD880007D02202120E06D0220E009A04D0042206
:10AD980002E0012200E002228918081A02B0F0BD80
:08ADA800FFFEFEFE80808080AA
:10ADB000F0B583B0002200295DD00378002B5AD073
:10ADC000032302469A4300240194E4438507ED0ED1
:10ADD000AC40E443156825430290044600931C40B0
:10ADE0006418042C2FD32748274FE9190646AE4391
:10ADF0000E4228D15568211F04291ED3EE1903469F
:10AE0000AB43334219D1956821460839042916D33A
:10AE1000EB190646AE431E4211D1D56821460C39C6
:10AE200004290ED3EB190646AE431E4209D1103C4D
:10AE300015691032042CD8D205E0121D02E0083248
:10AE400000E00C320C46280601990ED02804000EB2
:10AE50000AD02802000E11D0280E009800D004203D
:10AE60000146A14203D203E00121A14200D32146C1
:10AE70000298101A4218104603B0F0BD0221A142F8
:0CAE8000F5D2F5E780808080FFFEFEFE2A
:10AE8C00002A03D0013A8B5C8354FBD17047C04637
:10AE9C0000220B0011001A00002A02D0013A815442
:04AEAC00FCD170471E
:10AEB000002A09D0884207D007D280188918524248
:10AEC0008B5C83540132FBD17047013A8B5C835415
:04AED000FBD17047FB
:10AED40002480068002800D101487047580F00203C
:04AEE400000000204A
:10AEE8007F2805D8034A125C0348405C104070472D
:0CAEF800002070476CC50008DDC3000896
:10AF04007F2805D8034A125C0348405C1040704710
:0CAF1400002070476CC50008DDC3000879
:10AF20000200000004000000080000001000000003
:10AF3000FDFFFFFFFBFFFFFFF7FFFFFFEFFFFFFF3F
:10AF400000000000040000000200000008000000F3
:10AF500001000000020000000400000006000000E4
:10AF6000080000000A0000000C00000010000000B3
:0CAF7000200000004000000080000000F5
:10AF7C0000000000000000000000000000000000C5
:10AF8C0000000000000000000000000000000000B5
:10AF9C00010000000200000003000000040000009B
:10AFAC000600000007000000080000000900000077
:10AFBC000000000000000000000000000000000085
:10AFCC00010000000200000003000000040000006B
:0CAFDC004AC1000808B00008E8AF0008F7
:10AFE800E9AE000841BD000817B8000805AF000821
:10AFF8004DBD000825B8000831BD0008E9B70008B4
:10B008004CC10008DCC30008DCC30008DCC300082E
:10B01800DCC30008DCC30008DCC30008DCC300088C
:10B02800DCC30008DCC30008FFFFFFFFFFFFFFFFD2
:10B03800FFFFFFFFFFFF000010C100088EC30008DC
:10B048005DBF0008ABC30008B4BF00087CC300089C
:08B0580085C30008BBBF00081E
:10B06000034C206804348047FBE7FCF73BFBFEE71A
:04B07000ECC5000823
:10B0740004480549884385460448804704480549EF
:10B084000160EBE70080002007000000E9B400083D
:08B0940008ED00E000000008D7
:10B09C00FEE7FEE7FEE7FEE7FEE7FEE7FEE7FEE77C
:10B0AC00FEE7FEE7FEE7FEE7FEE7FEE7FEE7FEE76C
:10B0BC00FEE7FEE7FEE7FEE7FEE7FEE7FEE7FEE75C
:10B0CC00FEE7FEE7FEE7FEE7FEE7FEE7FEE7FEE74C
:0CB0DC00FEE7FEE7FEE7FEE7FEE7FEE70A
:10B0E800F0B581B000904C000120640C0446054680
:10B0F800064610D10C04240E01D000240BE00C06E7
:10B1080005D44C0606D000242546264603E0002434
:10B11800254600E0044603231746DF41032F13D8D2
:10B128007F443F797F00BF4406010411002C02D000
:10B138000AE0002D08D10098006841618168182351
:10B14800994311438160002001B0F0BD002EF2D078
:02B15800FAE714
:0AB15A0080B5806A00F00FF880BD98
:10B1640080B5806A816D40220A438265C16D0422E4
:0AB174000A43C26500F001F880BD37
:02B17E00704718
:02B18000704716
:02B18200704714
:0AB1840000690840411E8841704731
:02B18E00704708
:10B19000F0B583B004462820205C012802D10220AB
:10B1A00003B0F0BD264628360220707001200090C2
:10B1B0003070002A487806D0CA7812040002871836
:10B1C000887802903AE0C20603D5EF2210400A3098
:10B1D0004870CA78002713460A3B3D4608D3DAB2C6
:10B1E000CD255543ED0A0A226A439A1A2D011035DE
:10B1F0001543EAB203460A3B02973D4608D3D8B24C
:10B20000CD254543ED0A0A206843181A2D01103553
:10B2100012040543E8B20702887803460A3B09D3C3
:10B22000D8B2CD254543ED0A0A206843181A2B01F0
:10B23000103302931743029A024302922068CA22F3
:10B2400042625322426209780191C16849061BD4C7
:10B25000C16880220A43C260F5F700F805462068FD
:10B26000C168490610D4F4F7F9FF401B7D21C900DD
:10B270008842F4D9032070702168CA68FF224A62AC
:10B280000021317003B0F0BD0299C9B20F4301999A
:10B290004903C02297430F4347602046F7F73CF825
:10B2A0002168FF224A620028EAD1009870700020CD
:06B2B000307003B0F0BD98
:02B2B6007047DF
:02B2B8007047DD
:02B2BA007047DB
:02B2BC007047D9
:02B2BE007047D7
:02B2C0007047D5
:02B2C2007047D3
:02B2C4007047D1
:02B2C6007047CF
:10B2C80030B5816ACA070CD18A0714D44A071CD43E
:10B2D8000A0724D4CA062CD48A0634D44A063CD495
:10B2E8004CE00122520403685C689443C26A22431A
:10B2F8005A608A07EAD50122120403685C689443FD
:10B30800026B22435A604A07E2D50122920403687D
:10B318005C689443426B22435A600A07DAD50122DB
:10B32800D20303685C689443826B22435A60CA065E
:10B33800D2D50122120303689C689443C26B22434E
:10B348009A608A06CAD50122520303689C6894430E
:10B35800026C22439A604A0610D50122130502683E
:10B3680054689C43456C2C4354609D4206D103238A
:10B378005B0554689C43836C23435360090607D5D7
:10B388000121C904026853688B43C06C184350609C
:02B3980030BDC6
:10B39A0030B580214158212918D102465632938A64
:10B3AA00002B13D0016802E05B1E1C040ED0148827
:10B3BA00002C0CD0CC692406F6D5046D25788D6254
:10B3CA00641C04651488641E1480EDE730BD0120F6
:10B3DA00C0058A6882438A600868402202430A607C
:02B3EA0030BD74
:10B3EC0010B584214158222901680FD102465E32E2
:10B3FC0053884C6A1C40836D1C801488641E148016
:10B40C009B1C83651288002A05D010BD8869082210
:10B41C0002438A6110BD0246843209235B010C6829
:10B42C009C430C608B680124A3438B600021C16694
:0AB43C002021116000F031F810BD6E
:10B4460010B5842141582229016810D102465E3286
:10B456005388496A1940836D19701188491E1180F5
:10B46600816D491C81651188002905D010BD886948
:10B47600082202438A6110BD014684310922520125
:10B4860003681C6894431C609A680124A2439A606E
:0EB496000022C26620220A6000F002F810BDFB
:02B4A4007047EF
:02B4A6007047ED
:10B4A80030B57C21415C012901D1022030BD014623
:10B4B8007C3124224A600268136814680125AC4371
:10B4C80014606C07A34313600022426610460A709A
:06B4D80020224A6030BD95
:02B4DE007047B5
:02B4E0007047B3
:02B4E200FEE783
:02B4E4007047AF
:02B4E6007047AD
:02B4E8007047AB
:10B4EA0008D1002806D1F54204D801D3002A01D197
:10B4FA006D0D09D10020C143090DC904F0BDF9D170
:10B50A001242F7D1640DF5D00020C143490549081C
:10B51A00A6E000206146F0BDF0B50127FF070E0046
:10B52A005E403E40B446BE0A4C18DD18F442D7D2FB
:10B53A00F542E4D2640DECD06D0DEAD06419C9026B
:10B54A003943460DC0023143DB023B43DB0A10B4E8
:10B55A008E4685B297B26F43140C6C433E0CA41905
:10B56A00260C2404BFB227439CB26C43A419190CBD
:10B57A006943250CA4B249190D04090C6419000C7D
:10B58A0095B245433E0C76193743BFB2360C150CBB
:10B59A004543AD19A6B2240CAD192E0437432E0C1F
:10B5AA0036199DB24543AD19ACB22E0C89191D0C42
:10B5BA0045436D182E04290C3443704680B295B267
:10B5CA0045433E0C76193743BFB2360C150C45433A
:10B5DA00AD19A6B2AD19240C2E0437432E0C361918
:10B5EA009DB24543AD19ACB22E0C89191D0C4543C9
:10B5FA006D182E043443290C75462D0C90B26843FD
:10B60A003E0C80190604BFB23E43070CA0B23F1895
:10B61A00120C6A43D019020C80B2240CA4189AB2F4
:10B62A006A43121914042043120C89181B0C6B4329
:10B63A00C91810BC01273D05294203D1B61940415A
:10B64A004941013CFF077D0D013D641B0BDB6D0089
:10B65A00AC4209DA240500254208BE41684161412D
:0AB66A0066463143F0BD54E74EE799
:10B6740030B581B06A4611700269002A17D018C823
:10B684000838A3423CD243695C1C4461D1544269EA
:10B69400002A35D081698A4232D1036A002B03D053
:10B6A40001690446984720460021416128E0C268A8
:10B6B400002A09D018C80838A34221D25D1CA5422B
:10B6C40000D10021D1541BE08268002A08D018C898
:10B6D4000838A34214D25D1CA5420ED0C9B20DE0B5
:10B6E400036A002B0CD006C80838914208D2694678
:10B6F400012204469847204602E000219B00D150D5
:0AB704000168491C016001B030BD6E
:10B70E0010B54269002A07D00446036A002B01D007
:0AB71E00216998470020606110BD0A
:10B7280070B514460D460646FFF7D0FB0146304675
:0AB738002A462346FEF742FA70BDD0
:0AB7420080B50068FFF7A5FA80BD8E
:10B74C00F0B581B0154604464068A268E768C01998
:10B75C00D61BB54204D22A46FFF792FB7D1909E0AD
:10B76C000F463246FFF78CFBB919AD1B60682A46B1
:0AB77C00FFF786FBE56001B0F0BDA9
:10B78600F0B583B016460D46C7680021019006E065
:10B796000299C760361B2D196118002E1ED0029122
:10B7A6000269F943BA4202D95418816802E0521874
:10B7B600816854184268C91B8C4200D30C46B442B7
:10B7C60000D33446D01929462246FFF75CFBE71919
:10B7D600019881688F42DBD10027D9E7084603B07C
:02B7E600F0BDB4
:10B7E80010B50446002000290DD0002A0BD0097896
:10B7F80048B2002808D4002C00D02160002119602C
:0EB808005960411E884110BD0120C04310BD93
:0EB81600014641391A2901D22021084370470A
:0EB82400014641391A2901D2202108437047FC
:10B83200010002000400060008000A000C001000CB
:06B8420020004000800020
:10B84800B0B50146806A826D50231A42826D06D0D7
:10B85800D20610D4006D426B08469047B0BD012156
:10B868004B021A4382650268D3681B059B0F05D0FB
:10B87800FCF7FAFAB0BDFFF77EFCB0BD837E002B63
:10B88800F6D113681B07F3D593685B070ED40346FC
:10B89800583354680C25AC435460FF2402341A68AA
:10B8A800A2430A431A60FCF7DFFAB0BD826D202379
:10B8B8001343836503465C33C26D0A431A60FCF781
:04B8C800D3FAB0BD42
:10B8CC00F0B584B00E46022141770468A1680125C9
:10B8DC002943A160016A01291DD002290ED0032938
:10B8EC0027D1002A00D10EE10395032511462940EA
:10B8FC00042A00D3DEE033460025EAE0510863D089
:10B90C000296039503260B46334001934B1E032BE3
:10B91C0021D200273AE097080FD00395032339462C
:10B92C0019400091791E03290296019353D20025E8
:10B93C0084E04577002004B0F0BD002103231A40B9
:10B94C00032A00D0AEE07218715C09025378C91852
:10B95C0021809178ABE0B1430027029E7388358833
:10B96C002D04EB182360F388B5882D04EB182360A5
:10B97C00738935892D04EB182360F389B5892D045F
:10B98C00EB18236010363F1DB942E7D1019900290D
:10B99C00029E16D0BB00F1184D88F35A1B045B199C
:10B9AC002360019B012B0CD01F46CB888D882D0466
:10B9BC00EB182360022F04D04B8909890904C9189C
:10B9CC0021601146039DA943D20700D19BE0490099
:10B9DC00715A218097E09F43002531460E78360638
:10B9EC004B781B049B198E7836029B19CE789B19C9
:10B9FC0023600B791B064E793604F3188E793602C8
:10BA0C009B19CE799B1923600B7A1B064E7A360450
:10BA1C00F3188E7A36029B19CE7A9B1923600B7B16
:10BA2C001B064E7B3604F3188E7B36029B19CE7B9D
:10BA3C009B19236010312D1DAF42CFD1009F002FD9
:10BA4C00029E26D0A900735C1B0671184D782D043C
:10BA5C00EB188D782D025B19CD785B192360012FC3
:10BA6C0017D00B791B064D792D04EB188D792D020F
:10BA7C005B19CD795B192360022F0AD00B7A1B0658
:10BA8C004D7A2D04EB188D7A2D025B19C97A591851
:10BA9C0021601146019B9943039D03231A40032AFD
:10BAAC0000D150E7022A1ED0012A01D1715C21700D
:10BABC00046828E0AA430025334637682760776876
:10BACC002760B7682760F768276010362D1DAA42DB
:10BADC00F3D1002905D0AA001D469B5823600129EB
:10BAEC0009D1039D0FE072185278715C0902891814
:10BAFC002180046807E0AA18536823600229039D7B
:10BB0C0001D09168216021684577084604B0F0BDEA
:10BB1C00002A02D018228150704728228150704789
:10BB2C0042690B4693430A401104C918816170475E
:10BB3C0010B580214258212A0DD1034656331A885C
:10BB4C00002A026808D0016D0C789462491C0165CA
:10BB5C001888401E188010BD10688843106010684B
:08BB6C0040210143116010BDEE
:10BB740070B582B015460A4604460120C143DE1E54
:10BB84008E4200D318460090022D01D3092100E013
:10BB94000A2108180190069920462B46F8F7D8F890
:10BBA400262000212154A184E16121841C34A17147
:04BBB40002B070BDAE
:04BBB800007D704755
:08BBBC0080B5F9F7E9FF80BD37
:0CBBC40080B501204002F5F79FFE80BD17
:10BBD00010B582B00B4601AC2070012120460A4608
:10BBE00000F008F8002802D0207802B010BDC04351
:04BBF00002B010BDD2
:10BBF400F0B581B01E4615460C4607461846FEF7BA
:10BC0400F7FF0146002000290AD46543A54207D363
:10BC1400304639462A46FFF792FD2146FDF740FF9C
:04BC240001B0F0BDBE
:04BC2800C80F70478A
:10BC2C00F0B581B01C4615460091CA0017183E4667
:10BC3C00103EB068F1682A46FFF76DFC0CCEFDF79C
:10BC4C00EBFB009A032A0DDB183F561E2A462346AF
:10BC5C00FFF761FC0CCF083FFDF7DEFB761E083FBB
:10BC6C00012EF3D82A462346FFF755FC01B0F0BD50
:10BC7C00F0B581B01D4616460346C800022916DBF6
:10BC8C0000931F18083F4C1C304629460CCF083F28
:10BC9C00FDF7C2FB32462B46FFF73DFC641E083F06
:10BCAC00022CF3D8009B083306460D4600E01B1807
:10BCBC00083B0CCB30462946FDF7AEFB01B0F0BD7E
:08BCCC00C1174840401A7047FF
:10BCD40070B5012A09DB0C460546561C2846214648
:0CBCE400FFF7C6FC761E012EF8D870BDDC
:10BCF00070B50446C80610D4880503D53025012A3E
:10BD000003DA70BD2025012A07DB561C2046294690
:0CBD1000FFF7B0FC761E012EF8D870BDC5
:10BD1C0010B50C46436A01212046FFF765FF10BDA4
:04BD2C0040207047FC
:10BD3000024601207F2901D9C04370471170704726
:0CBD4000014661391A2900D220387047F2
:0CBD4C00014661391A2900D220387047E6
:0FBD580049205265666572656E7A3D25660A0060
:0BBD6700547368756E743D25660A0079
:10BD72002D2D2D204761696E20447269667420431F
:07BD8200414C202D2D2D0086
:0FBD890041637475616C20543D256620430A00A8
:10BD980041637574616C20493D25662041287769A7
:10BDA80074686F7574206761696E2074656D7020A2
:10BDB800647269667420636F7272656374696F6E0A
:03BDC800290A0045
:10BDCB004B6F7272656B74757266616B746F723DDB
:10BDDB002566205B2031202F2043656C73697573BA
:03BDEB005D0A00EE
:10BDEE004552524F52204144535F313236305F53E9
:0BBDFE0065744461746152617465005B
:10BE09004552524F52204144535F313236305F53CD
:0BBE1900657443686F704D6F64650036
:10BE2400454550524F4D20776173206368616E67BA
:10BE3400656421205765206E65656420746F2070E9
:10BE4400726573657276652063616C696272617490
:10BE5400696F6E20616E642073657474696E6773B4
:07BE640020646174612100FC
:10BE6B00454550524F4D20464143544F5259205255
:0FBE7B004553544F52452F5550444154452100D3
:0FBE8A007265616420636F6E6669672E2E2E00ED
:10BE9900666163746F727920726573746F72652E4F
:03BEA9002E2E003A
:10BEAC0050524F54454354494F4E3A204F425F52E3
:0BBEBC0044505F4C4556454C5F32007F
:10BEC70050524F54454354494F4E3A204F425F52C8
:0BBED70044505F4C4556454C5F310065
:10BEE20050524F54454354494F4E3A204F425F52AD
:0BBEF20044505F4C4556454C5F30004B
:10BEFD00466C61736820756E6C6F636B2065727232
:03BF0D006F720050
:10BF10004F5554505554535F4C56505F5348554EEF
:10BF2000545F554E44455254454D50455241545529
:03BF300052450077
:10BF33004F5554505554535F4F56505F5348554EC9
:10BF4300545F554E44455254454D50455241545506
:03BF530052450054
:07BF5600286E756C6C2900D8
:10BF5D004A616E75617279004665627275617279BA
:10BF6D00004D6172636800417072696C004D6179BA
:10BF7D00004A756E65004A756C7900417567757379
:10BF8D00740053657074656D626572004F63746FF4
:10BF9D00626572004E6F76656D6265720044656311
:07BFAD00656D626572000082
:07BFB400414D00504D00005B
:0FBFBB0025612025622025652025542025590069
:10BFCA004552524F52205452494D4D494E472056E0
:06BFDA00414C55455300E7
:0EBFE00075617274206572726F72200A0D0016
:10BFEE002D2D2D204761696E202043414C202D2D93
:02BFFE002D0014
:0AC0000054736869703D25660A005C
:10C00A002D2D2D204761696E202043414C20454E3D
:06C01A0044452D2D2D0010
:0EC0200064656C746120543D256620430A005F
:0AC02E0052656620493D25660A00B0
:10C038004552524F52204144535F313236305F49A6
:0EC048006E7075744D757853656C6563740089
:10C0560046697273742073746172742064657465C2
:06C0660063746564210013
:0EC06C004953454E534F523A20496E697400B5
:10C07A002E2E2E466C61736820756E6C6F636B652D
:02C08A00640050
:10C08C00466C617368206F6220756E6C6F636B20F9
:06C09C006572726F720074
:0EC0A200466C61736820206C6F636B656400F0
:10C0B0004F5554505554535F4C56505F5348554E4E
:10C0C000545F4F56455254454D5045524154555278
:02C0D000450029
:0EC0D2004F5554505554204C5650204F4B00A3
:10C0E0004F5554505554535F4F56505F5348554E1B
:10C0F000545F4F56455254454D5045524154555248
:02C100004500F8
:0EC102004F5554505554204F5650204F4B006F
:10C1100053756E646179004D6F6E6461790054757A
:10C120006573646179005765646E65736461790055
:10C13000546875727364617900467269646179004C
:0AC1400053617475726461790000A8
:02C14A004300B0
:02C14C002E00C3
:10C14E004672657175656E6379204D6561737572A2
:09C15E006564203D2025640A00FF
:10C16700492028776974686F757420636F6D7065EF
:0DC177006E736174696F6E293D25660A00C4
:10C184004144535F313236305F4261747465727971
:10C1940043757272656E744761696E43616C69625E
:10C1A400726174696F6E53746172743A20455252AD
:10C1B4004F5220494E2043414C4942524154494F29
:10C1C4004E2C204E4F205245464552454E43452065
:09C1D40043555252454E5421001E
:10C1DD004E6F726D616C2073746172742077697427
:10C1ED00686F757420454550524F4D206368616EE0
:0DC1FD006765732064657465637465640094
:10C20A00454550524F4D2046554C4C2052455354AB
:05C21A004F5245210018
:10C21F00454550524F4D2053544F524520434F4E9A
:05C22F00464947210013
:0DC234004144533132363020496E697400A8
:10C241002E2E2E466C617368206F6220756E6C6FA6
:05C25100636B65640051
:10C256002E2E2E44697361626C65206C6F636B20B1
:10C2660070726F636573732066696E69736865645F
:01C2760000C7
:10C27700466C617368204F7074696F6E627974657C
:10C287002070726F6772616D6D206661696C65649D
:01C2970000A6
:10C298002E2E2E466C617368206C6F636B20616C68
:0DC2A80072656164792061637469766500D8
:10C2B5002E2E2E456E61626C65206C6F636B20655A
:05C2C50072726F7200AF
:10C2CA004F5554505554535F4C56505F434849504C
:10C2DA005F4F56455254454D50455241545552456B
:01C2EA000053
:10C2EB004F5554505554535F4C56505F4241545424
:10C2FB004552595F554E444552564F4C5441474554
:01C30B000031
:10C30C004F5554505554535F4F56505F4348495006
:10C31C005F554E444554454D504552415455524538
:01C32C000010
:10C32D004F5554505554535F4F56505F43484950E5
:10C33D005F4F56455254454D504552415455524507
:01C34D0000EF
:05C34E002D494E4600E0
:05C353002D696E66007B
:05C358002B494E4600D8
:05C35D002B696E660073
:10C3620000000000000054545220524547474553F4
:01C3720000CA
:09C373005465726D696E616C0085
:09C37C00256D2F25642F257900A1
:09C3850025483A254D3A255300E4
:10C38E0053756E004D6F6E005475650057656400F1
:0DC39E005468750046726900536174000018
:10C3AB004A616E00466562004D6172004170720019
:10C3BB004D6179004A756E004A756C0041756700D6
:10C3CB00536570004F6374004E6F760044656300D5
:01C3DB000061
:01C3DC000060
:0DC3DD0000070320041702010857104080DC
:04C3EC00AD85000813
:10C3F00056616C7565206E6F742076616C6964009F
:10C400004B6F7272656B74757266616B746F723D9F
:04C4100025660A0093
:10C414002D2D2D204761696E204472696674204376
:0CC42400414C20454E4445202D2D2D009C
:10C430004552524F52204144535F313236305F53A0
:10C440006574496E7465726E616C5265666572657D
:04C450006E636500B2
:0CC4540057726974696E6720534E210016
:10C46000554E4B4E4F574E20434F4D4D414E44007D
:10C47000466C617368204F7074696F6E6279746581
:0CC480002070726F6772616D6D65640062
:10C48C00537461727420656E61626C6520726561B3
:10C49C00646F75742070726F74656374696F6E006D
:10C4AC002E2E2E466C61736820756E6C6F636B005C
:10C4BC00466C617368204F7074696F6E6279746535
:08C4CC00206C6F636B656400D6
:10C4D4002E2E2E456E61626C65206C6F636B20702E
:10C4E400726F636573732066696E6973686564004F
:10C4F4004F5554505554535F4C56505F4F56455208
:08C5040043555252454E54000C
:10C50C004F5554505554535F4F56505F4F564552EC
:08C51C0043555252454E5400F4
:10C524004F5554505554535F4F56505F42415454E5
:10C534004552595F4F564552564F4C54414745005A
:10C544003031323334353637383941424344454645
:10C554003031323334353637383961626364656675
:04C564004E414E00F6
:04C568006E616E0092
:10C56C002020202020202020206828282828202057
:10C57C0020202020202020202020202020202020AF
:10C58C004810101010101010101010101010101067
:10C59C008484848484848484848410101010101007
:10C5AC001081818181818101010101010101010160
:10C5BC000101010101010101010101101010101014
:10C5CC001082828282828202020202020202020231
:10C5DC0002020202020202020202021010101020D9
:10C5EC0039C6000829000020211400004BC60008A1
:10C5FC00000000200CC60008290000006BB00008E9
:10C60C00DCAF0008DCAF0008DCAF0008DCAF0008D2
:10C61C00DCAF0008040000004C0F0020500F00207D
:0CC62C00540F00200024F4000100000066
:10C63800206861680834002200E042540139FCD5C2
:02C64800704739
:10C64A0020686168A2680C3401E08B5C8354013A6B
:04C65A00FBD5704755
:020000040801F1
:04C7FC00A86081535D
:040000050800B075CA
:00000001FF
